:10000000F01F001045380000413800004138000062
:100010004138000041380000413800000000000075
:100020000000000000000000000000004138000057
:100030004138000000000000413800005516000063
:1000400025140000251400002514000025140000CC
:1000500025140000251400002514000025140000BC
:1000600025140000251400002514000025140000AC
:10007000251400003D3800003D3800003D380000E8
:100080000D170000251700003D1700005517000050
:100090003D3800001D1800003D3800003D380000CC
:1000A0003D3800003D3800003D3800003D3800007C
:1000B0003D3800003D3800003D3800003D3800006C
:1000C00008B500230B60036000F01AFE08BD08B5F8
:1000D0000A20002101F0BAFA08BD000038B5094B2A
:1000E0000D1C041C1968012001F060FB012001F0C7
:1000F0003DFB291C201C02F023FF012001F046FBE0
:1001000038BDC046BC04001070B5054E051C0E2459
:10011000013C295D301C01F09DFD002CF8D170BD23
:10012000743A000038B5164801F094FD154C201CB7
:10013000FFF7EAFF144D4221281C01F08BFD201C23
:100140000E30FFF7E1FF4321281C01F083FD201C46
:100150001C30FFF7D9FF0D4801F07CFD201C2A3030
:10016000FFF7D2FF281C4E2101F074FD201C38300F
:10017000FFF7CAFF616D064801F06CFD38BDC0464F
:10018000773A0000C40400107D3A0000843A000071
:100190008A3A000010B5084B041C1968012001F0D0
:1001A00005FB012001F0E2FA201C02F059FE0120BB
:1001B00001F0ECFA10BDC046BC04001008B50020E8
:1001C000FFF7E8FF08BD000008B5021C024903481C
:1001D00001F040FD08BDC0469E3A0000963A00007E
:1001E00013B59620000201F057FB00F015FC1548EE
:1001F00000210322144B00F003FD00F017FCFFF771
:10020000DDFF1248FFF7E0FF002401F0E3FB0028C8
:1002100003D001F021F8002409E00A2001F046FA99
:10022000684601A9FFF74CFF009B002B03D1084B48
:1002300001349C42E9DDFFF7C1FF064801F00AFDE9
:1002400013BDC046A53A000000000010B43A0000FB
:100250006F170000BA3A00007047000073B5124BE8
:10026000041C1249186803F06FFB11490090114AF1
:10027000114B201C01F0F9FC00F024FE002812D0E4
:1002800000F03CFEFA218900051C03F05DFB061C12
:10029000201C01F037FD094B201873430849EB1867
:1002A000321C01F0E2FC73BDC004001040420F009C
:1002B000C53A00009E3A0000D23A000018FCFFFF49
:1002C000D63A000070B5051C0C1C161C00F0A4FBEF
:1002D000291C201C0022064B00F092FC301C01213E
:1002E0000922044B00F08CFC00F0A0FB70BDC0465E
:1002F000000000100C00001000B5084B89B01A78FF
:10030000074B68461B78074901F0AFFC694601209E
:10031000054AFFF7D7FF09B000BDC046C80100106D
:1003200008000010E13A0000EF3A000073B5264BD8
:1003300000241D78254B1E78FFF7DEFFFFF73EFFF8
:10034000684601A9FFF7BCFE009B002B26D0182BA6
:1003500031D004DC142B0ED0152B1AD106E0352B2E
:100360000BD0842B2DD0342B13D10CE0164B1A78E4
:100370003E2A0ED805E0144B06E0144B1A78062AE4
:1003800007D8013204E0114B1A78002A01D0013A53
:100390001A7000F02DFBFFF7AFFF0024009B002B2D
:1003A00002D0C82001F082F904200121013401F0BB
:1003B0004DF91D2CC4DD044B1D70044B1E7000F064
:1003C00017FBFFF7FBFE73BDC8010010080000100B
:1003D00010B590B0041C6846FFF740FF69466A46B6
:1003E000201CFFF76FFF10B010BD000073B5182080
:1003F0000021FFF773FE4B4E4B4D00249836012031
:1004000001F0C4F9002C01D0002000E006200121F9
:1004100001F01CF9684601A9FFF752FE009B002B72
:1004200021D1002CF0D13368002B0DD03F4B00942C
:100430001A6811321A6004E002F0BCFC009B013320
:100440000093009B102BF7DD394BED18DED51820FB
:100450000021FFF743FE334B94331C6863425C4139
:1004600000F08EFACEE7002C06D0182BC7D1314809
:10047000FFF7AAFE00F0E2FA009B182B36D1019B91
:1004800000220192822B25D004DC322B11D0732B59
:100490002BD11CE0872B20D0C22B02D0832B24D160
:1004A0000DE0254B19680131196002291ED11A602F
:1004B0001CE0224B01201B68C01A00F045FD012002
:1004C000FFF786FFFFF77AFEFFF701FE0EE0FFF76A
:1004D00087FE0BE0FFF72AFF08E0194B1A70194B53
:1004E00005221A7000F084FA00E0019300F018FD74
:1004F000154B0120196801F059F9012001F036F976
:100500000098019902F01CFD064B94331B68002BE8
:1005100003D100F035FA012402E003F02DF90024A4
:10052000014D6CE7C404001020BF0200F802001067
:100530000CFEFFFF033B0000A0010010180000109C
:10054000C801001008000010BC04001013B501F031
:1005500009FC00F0A1FB00F071FA00200421012247
:1005600000F0A2FE0020021C042100F0EBFE00209F
:100570000521012200F098FE0020021C052100F058
:10058000E1FE1348002100F001FF0021114800F0B6
:10059000FDFE00F027FC00F06BFE2824201CFFF776
:1005A00017FF023CFA2001F081F8022CF6D101F08D
:1005B00021FC02F025FB1E2300930F230193064824
:1005C00006490022064B02F0CDFBFFF70FFFC046A5
:1005D000984004409C400440F9370000C1000000EE
:1005E000F802001000B500E001300378202BFBD0AA
:1005F00000BD00B5031C303BDAB2092A01D8181C33
:1006000008E020231843031C613B5738052B01D910
:100610000120404200BD70B50E1CFFF7E3FF00252E
:10062000041C06E0FFF7E5FF002805DB2D0105436C
:10063000013420780028F5D13560201C70BD000001
:1006400008B500F05BFC011C014801F003FB08BD8C
:100650000D3B000000B5C300181A064BC018072355
:10066000013BC25C002A03D1002BF9D1012000E03C
:10067000002000BD600500107FB5194801F0EAFABE
:1006800000250326354219D1281CFFF7E3FF002877
:1006900010D0681CFFF7DEFF00280BD0A81CFFF766
:1006A000D9FF002806D0E81CFFF7D4FF002801D0AE
:1006B00004350FE00B48291C01F0CCFA291C6846D0
:1006C00001F0BCFB6846FFF71FFD074801F0C2FAC6
:1006D0006C1C251CFF2DD5DDFFF724FD7FBDC0461A
:1006E000193B00001E3B0000D77C000070B50E1CBB
:1006F000FFF778FF0D25041C2078FFF77AFF00280C
:1007000007DB01347055013DF6D2201CFFF76AFF6C
:1007100000E0002070BD000030B5464C87B0236873
:100720000868002B06D1444801F094FA02F068FAF8
:10073000012357E0012B12D10379202B07D0002B86
:1007400005D03E49042201F0F0FA002803D1394BCC
:100750001A6801326AE03A4801F07CFA5EE00378F8
:10076000412B1BD1374C0230211CFFF7BFFF002863
:1007700054D00378422B51D1211C02300E31FFF7A7
:10078000B5FF00284AD00378432B47D1211C023003
:100790001C31FFF7ABFF002849D13FE04D2B23D19F
:1007A000294D0230291CFFF7A1FF002836D003781D
:1007B0004E2B33D1291C02300E31FFF797FF002852
:1007C0002CD00378472B29D1023005A9FFF723FF4E
:1007D000059B002B22DB2A3D6B651C481C4901F060
:1007E00039FA0023236022E005A9FFF714FF0378FC
:1007F000041C202B01D0002B10D10025201C01A9A6
:10080000FFF774FF0599041C691801A801F02AFB81
:10081000002C03D00135042DF0D108E002F0F0F9EE
:100820000A480C4901F016FA024B00221A6007B080
:1008300030BDC046D0020010273B0000193B00002D
:100840003D3B0000C4040010EE040010493B0000D2
:10085000533B0000563B000037B54C6824E0201C99
:10086000FFF7C0FE01A9FFF7D6FE019B041C002B79
:100870001DD0D8B2FF2B09DD00F0DEF9051C019870
:100880000012C0B200F0D8F9019003E000F0D4F9F2
:10089000002501900198002802D0291CFFF71EFCBA
:1008A00023785A1E9341E4182378002BD7D137BD03
:1008B00008B5064A012113784B40137001D0044952
:1008C00000E00449044801F0C5F908BDB103001077
:1008D0000A3B00005D3B0000613B000070B5051C59
:1008E00001200821021C00F02DFD07240126012013
:1008F0000821002200F026FD2A1C2241324000205F
:10090000022100F01FFD01200821021C00F01AFD49
:10091000013CECD270BD10B50021041C0A1C022061
:1009200000F010FD201CFFF7D9FF10BDF7B5012323
:1009300000930023019372B66C46061C02AF01CCF3
:1009400050235B421843C0B2FFF7E5FF0020FFF7DA
:10095000E2FF1020FFF7DFFFE020FFF7DCFF0025BC
:1009600002200021012200F0EDFC705D0135FFF74F
:10097000B5FF842DF4D18436BC42E0D162B6F7BD18
:1009800008B5AC20FFF7C7FFAE20FFF7C4FFA520D6
:10099000FFF7C1FF08BD38B50D1C041C012200F093
:1009A00083FC291C201C012200F0CCFC38BD08B5BA
:1009B000AF20FFF7B0FFA420FFF7ADFF08BD08B5DB
:1009C000AE20FFF7A8FF08BD10B5041CF820FFF704
:1009D000A2FF201CFFF79FFF10BD10B5041C812053
:1009E000FFF799FF3F202040FFF795FF10BD000063
:1009F00008B5074B20201B781843FFF78CFF0A200F
:100A000000F054FE034B1878FFF7E7FF08BDC0461F
:100A100008000010C801001008B584220248002117
:100A2000520001F04FF908BDB203001008B50248AA
:100A3000FFF77CFF08BDC046B203001008B50120D7
:100A40000821FFF7A8FF00200221FFF7A4FF0220E2
:100A50000021FFF7A0FF02200621FFF79CFF0320E3
:100A6000011CFFF798FF0320011C002200F06AFC24
:100A700002200621002200F065FC0621012202204E
:100A800000F060FCFFF7C8FFFFF7D0FFA220FFF7E0
:100A900042FFA020FFF73FFFC020FFF73CFF0020F0
:100AA000FFF792FF0A2000F001FE4020FFF733FF1E
:100AB0002C20FFF730FF322000F0F8FD2E20FFF74A
:100AC0002AFF322000F0F2FD2F20FFF724FF0A203A
:100AD00000F0ECFDFFF78CFFAF20FFF71CFFA42018
:100AE000FFF719FF08BD000000B50F290ED88328B5
:100AF0000CD8CB08842253430722C0181140044B62
:100B000080220A41111C1A5C1143195400BDC046D1
:100B1000B2030010F0B55B18DBB216E08425CC08F8
:100B20006C4307270F40802504193D41EFB2A618FA
:100B30009C4605E0064BE5182B7801343B432B70AF
:100B4000B442F7DB01316346C9B29942E6D3F0BD46
:100B5000B2030010F0B589B0059106921C1C5D68C7
:100B6000DB78834202D22478039444E0A378234ABA
:100B7000C01A0023954209D14300181803234519D0
:100B8000039309E02A7801330232AD188342F9DB7E
:100B900069782B7803910235EB18002604930196AF
:100BA00025E0082F05D1049A954224D02E780027FD
:100BB0000135F30706D5029A069B0798D118C9B2EA
:100BC000FFF792FF0299761001310291013707E099
:100BD000002202920199059A08278B18DBB207932D
:100BE000637802999942DCDB019A01320192019B00
:100BF00003998B42ECDB039809B0F0BD703B000019
:100C0000F0B585B0061C0C1C0292039301F07AF833
:100C100000250190832708E0705D211C029A039B48
:100C2000FFF798FF013024180135A74202D3019B3A
:100C30009D42F1D305B0F0BD00B50F230209184065
:100C40008000031F00D52833002B0EDB511E03202C
:100C5000884280414042002807D1242B06DC042131
:100C60008A1A0349CB18985C00E0002000BDC046FA
:100C7000223F000070B5064E051C0024A05D054B08
:100C8000291CC018013400F081FB0A2CF6D170BD7C
:100C90005E3F000000400440F8B51020FFF7EAFF77
:100CA000094C271C143725786678281C311C002233
:100CB00000F0FAFA0234281C311C012200F042FB39
:100CC000BC42F0D1F8BDC0464A3F0000F8B50B4C1D
:100CD000271C143725786678281C311C012200F067
:100CE000E3FA0234281C311C002200F02BFBBC422A
:100CF000F0D10020FFF7BEFFF8BDC0464A3F00001C
:100D0000F0B589B0002404900591FFF7C5FF0220DB
:100D1000072101220694079400F0C6FA0220072159
:100D2000221C00F00FFB201C0B2100F0E1FAA04276
:100D300002D11823069301240021264D03916A78DD
:100D40002F78111C0192381C012200F0ADFA381CDA
:100D50000199002200F0F6FA03231F4E029314E0DB
:100D60003078717800F0C4FA002807D103991B4A43
:100D7000A3008A5C183369465A500134029A039BD7
:100D8000013A013302920393023EE30F0021012254
:100D9000A2424B41DBB28B4202D0029B8B42DFDA94
:100DA000381C0199002200F07FFA0199381C0122B9
:100DB00000F0C8FA0A4902358D42C0D1201E06D083
:100DC000069B049A05991360079B01200B6009B0EC
:100DD000F0BDC0464A3F0000203F0000223F000017
:100DE0005E3F000008B50120021C0B2100F05CFAF8
:100DF00001200B21002200F0A5FA0320022101228C
:100E000000F052FA03200221002200F09BFA08BDF4
:100E100037B5234B10211A68051C8A431A60214BF1
:100E20008022196892010A431A6001200B210022D6
:100E300000F03AFA01200B21002200F083FA1A4B4D
:100E40009F211A68194C8A431A601A6818491A6057
:100E5000184B186802F078FD8023000218432A1C02
:100E600020600221032000F06DFA142000F01EFC27
:100E70002368FF229343236023680F4A13432360B0
:100E80000E4B1A680192019A002AFADA22680C4B7A
:100E900013402360FFF7A6FF01980004800D3EBDBC
:100EA00038820440808004409840044000C00140E3
:100EB00000093D00C0040010800000012CC001406A
:100EC000FFFFFFF810B50C4C2068002813DA002053
:100ED0002060FFF79DFF0A280ADC0120FFF798FF3A
:100EE0000138C023FF385B00984201D801232360FA
:100EF000FFF778FF206810BD1400001008B5FFF759
:100F0000E1FF011E08D00120FFF782FF011E03D080
:100F1000024802F019FD011C081C08BD50BB12005C
:100F200008B5FFF7CFFF00280AD0FFF7E7FFFA2246
:100F3000031C0021C00FD2009A424841014B1860A7
:100F400008BDC046CC01001010B500280DD0254BBF
:100F500080211A688A431A60234A012311681942C2
:100F6000FCD0224B03221A6001E0204B1860204B7A
:100F7000012200211A6019601A6019681142FCD020
:100F80001C4B01221A601C4A80211468490221432B
:100F900011601A1C002804D1124B802419682143C7
:100FA0001960164B196888421AD01860002801D0C1
:100FB000134800E01348116802F078FC124C21211C
:100FC000206002F0C1FC114B18609620000200F076
:100FD00063FCFA212068890002F0B6FC00F04CFBAB
:100FE00010BDC046388204400C800440708004402C
:100FF0007480044078800440808004401800001011
:10100000006CDC02001BB700C0040010BC04001020
:1010100008B500F03BF9134B00211A68120B1203BC
:101020001A60114B1A68120B12031A600F4B1A68E0
:10103000120B12031A600E4B1A68120B12031A607D
:101040000C4B012219600C4B1A6019601A60196868
:101050001142FCD0094B23221A600120FFF774FFD4
:1010600008BDC04600800050008001500080025042
:1010700000800350408004404480044008800440C5
:1010800070B50F490F4800F0E5FD0F4800F0E2FD94
:101090000E4E0F4D00242B196159DA68301C0A4B93
:1010A000143400F0D7FD782CF5D10A4800F0D2FDB9
:1010B00000F018FB011C084800F0CCFD70BDC046D4
:1010C0009E3A0000683F0000BA3F00007A3F0000EF
:1010D0001C000010853F0000A73F0000F0B53C4B0E
:1010E0008BB01D68002D3AD03A4B02901B6801204E
:1010F0009B685DE001342378202BFBD0002B3AD095
:10110000B30008336A469C500136FF2D01D135E00B
:1011100001342378202B01D0002BF9D1202B02D1D0
:10112000002323700134012E1BD12A4F2A4B0722A2
:101130003B6001923D1C09E02B680298196800F0A1
:1011400003FE002808D02B6814332B60019B013B61
:101150000193002BF0D132E03B681D7901E0041CC3
:101160002E1C2378002B06D000230722B2425B41BD
:10117000DBB2002BBFD1002E1CD000E00025154CA7
:10118000022E05D10398154900F0DEFD002801D09C
:10119000AE420AD823681248D96800F05BFD236884
:1011A0001048196900F056FD04E02368F0B29B680E
:1011B00002A99847064B1B68002B07D103E0019852
:1011C000011CFFF75DFF084800F044FD0BB0F0BDC7
:1011D000D0020010D80200101C000010B43F000024
:1011E000B63F00004E3B0000BD3F000038B5041C78
:1011F000154D0A2808D002D808281CD110E00D2867
:1012000002D07F2817D10BE02B6800221A700F48FC
:1012100000F020FD0E4C201CFFF760FF2C6012E058
:101220002A680B4B9A420ED90A48211C00F012FD85
:101230002B68013B06E00748211C00F00BFD2B68E2
:101240001C7001332B6038BDD4020010BA3F00007F
:10125000D0010010C93F000008B503E000F098FB82
:10126000FFF7C4FF00F0B6FB0028F7D108BD00006F
:1012700008B5034A034B04481A6000F0EBFC08BDB4
:10128000D0010010D4020010BD3F0000044B4021EB
:101290001A680A431A60034B01221A707047C0464D
:1012A00080800440DC02001070B50E4B061C1B78D9
:1012B0000D1C141C002B01D1FFF7E8FF013E022E8C
:1012C00003D8094BB600F35800E0084B1A68012C0C
:1012D00003D1AC4014431C6003E00124AC40A243A2
:1012E0001A6070BDDC0200104C400000008000500D
:1012F00038B50F4B051C1B780C1C002B01D1FFF7D8
:10130000C5FF0020032D11D8281C012302F0BAFAD2
:1013100002040608074A04E0074A02E0074A00E020
:10132000074A1068A3401840431E984138BDC04684
:10133000DC020010FC3F0050FC3F0150FC3F02501B
:10134000FC3F035070B50E4B061C1B780D1C141C83
:10135000002B01D1FFF79AFF013E022E03D8094B63
:10136000B600F35800E0084B1A68012C03D1AC40DA
:1013700014431C6003E00124AC40A2431A6070BD1A
:10138000DC02001058400000FC3F005038B5084B0C
:10139000041C1B780D1C002B01D1FFF777FF23687D
:1013A00018229343236023681D43256038BDC0463F
:1013B000DC0200101F234209184001238340181C3F
:1013C000014B9200D050704700E100E01F2342091A
:1013D000184001238340181C2032024B9200D05049
:1013E0007047C04600E100E0054B3F221A60054B04
:1013F00001221A60044B40211A688A431A60704720
:1014000024800440D88004403882044008B5044B4E
:1014100040211A688A431A60FFF7E6FF08BDC046FC
:101420003882044008B5154B1868FFF78DFD07207A
:10143000FFF7CCFF0820FFF7C9FF0A20FFF7C6FF20
:101440000C20FFF7C3FF0B20FFF7C0FF0920FFF7B9
:10145000BDFF0B4A0023136001210A4A4942116073
:10146000094A1360094A1360094B01221A60094BAB
:101470001A6801321A60C04608BDC0461800001044
:10148000048204400882044004C000403CC0004084
:1014900000C00040E002001008B5FFF717FC0A4842
:1014A0000021FFF773FF09480021FFF76FFF08488D
:1014B0000021FFF76BFF07480021FFF767FF064891
:1014C0000021FFF763FF08BD0840044000400440CE
:1014D000AC400440144004401C400440F8B5071CD4
:1014E0000C1C72B6FFF7D8FF434B1A68434B1A60C7
:1014F000002F01D0424B00E0424B434A04211360CD
:10150000424B434D1A680A431A6000232B609C42E9
:1015100018D00720FFF74EFF0820FFF74BFF0A20E7
:10152000FFF748FF0C20FFF745FF0B20FFF742FFB6
:10153000384B394A19680A401A602A68EC235B0163
:1015400013432B60002F4FD0344B354C35490026C8
:101550000E60201C1E60311CFFF718FF301C092193
:10156000321CFFF7A1FE301C0921321CFFF7EAFEF6
:101570002D4B8022196811431960236807218B4382
:101580002360236802210B4323607B00DB19990150
:101590005B189B002549DF19254B0F60032119605B
:1015A000244B2549186801401960196809200A432D
:1015B0001A60FFF7FFFE174A802311689B0019434A
:1015C00011602A68022113431C4A2B600123136017
:1015D0001B4A11601B4A13491360166013601068A0
:1015E0001842FCD001230B60174B012252421A60B3
:1015F00062B630BFF8BDC046388204403482044031
:10160000BF180000FF1800003082044010ED00E019
:1016100004820440008204407FE2FFFF0440014056
:101620006440044004C000408080044018C0004072
:1016300014C000403CC000400FF0FFFF7880044021
:1016400070800440748004400882044008B5FFF7AD
:1016500045FF08BD00B5064B1A6801321A601B68C9
:10166000013303D1034B1A6801321A6000BDC04632
:10167000E8020010E402001000B5074B98420AD8B7
:10168000064A00231360064A01381060054A1360B9
:10169000054B07221A6000BDFFFFFF00E8020010A3
:1016A00014E000E018E000E010E000E000B50C4AB3
:1016B0001368002800D10120C1438B4204D809E0FF
:1016C00011688142FCD301E0591C08181168994245
:1016D000F6D203E01168C91A8142FBD300BDC046AF
:1016E000E802001010B5064BFA211868054B890076
:1016F0001C6802F0DBF8044B5C43201810BDC046A8
:10170000E8020010E402001037894100034B012277
:101710001A60034B1A6801321A60704700C000401B
:10172000EC020010034B01221A60034B1A680132CD
:101730001A60704700000140F0020010034B0122C4
:101740001A60034B1A6801321A607047004001406A
:10175000F4020010034B01221A60034B1A68013295
:101760001A60704700800140F802001000B50028A0
:1017700003D1044B01221A6003E0012801D1024B7E
:10178000186000BD044001400480014000B50028FD
:1017900002D1044B186004E0012802D1024B002260
:1017A0001A6000BD044001400480014010B50028CB
:1017B0000FD1124B80221C68920022431A60104BFA
:1017C000032218600F4B19600F4B1A608022D2025F
:1017D00011E0012811D1094B80221868D200024380
:1017E0001A600A4B00221A60094B03221960094B48
:1017F0001A6080221203084B1A6010BD80800440DA
:10180000F40200101840014014400140F80200109A
:10181000188001401480014000E100E008B5184B39
:101820001A680E231340062B0DD1164B9E221B68FF
:10183000DBB2134204D0144A5360144B1B681EE001
:10184000D9071CD501E0042B05D1104B1868C0B294
:1018500000F0AFF813E00C2B06D10B4B8022596837
:1018600052000A435A600AE0022B08D1054B1A685D
:10187000054B910601D5002200E001229A6008BDC7
:101880000880004014800040FC02001000800040EE
:1018900000487047FC02001070B5294C294B80228B
:1018A0009203DA67061C0021201C902200F00AFA3D
:1018B0000023A360244B07251A68244CAA431A600E
:1018C0001968012211431960214B1968A943196055
:1018D0001968114319601F4B8021186849010143A1
:1018E00019601D4B1A608322226019681B4B18680F
:1018F00001F0DCFF311C000901F0D8FF1849030A90
:10190000184A0B60C0B2032310602360164B1D60A1
:10191000164B186860201C680440602CFBD101E065
:10192000146800E001201C680442F9D1044B012234
:101930001A700F4B802292031A6005230B6070BD52
:10194000FC02001004E100E0A44004400C800040D0
:10195000A84004408080044098800440C0040010E7
:101960000480004000800040088000401480004057
:1019700000E100E000B5044A202311681942FCD0C0
:10198000024B186000BDC04614800040008000403B
:1019900008B5FFF77DFF827B031C8218D07B9A7B02
:1019A0000132D2B29A7352B2002A01DA00229A733B
:1019B00008BD10B5041CFFF76BFF437BC318DC7335
:1019C000437B0133DBB243735BB2002B01DA0023AC
:1019D000437310BD08B5FFF75BFF827B437BD01AD2
:1019E000431E984108BD30B5002402E00570013463
:1019F00001301D5D002DF9D1121B131C02E0017096
:101A0000013B0130002BFADCD043C0170240A01884
:101A100030BDF8B5051C0F1C1E1C541E092B01D827
:101A200000240FE0181C0A2101F040FF221C031CB7
:101A3000391C281CFFF7EDFF041C2D1805E02F7042
:101A400001340135013A002AF9DC301C0A2101F089
:101A500071FF30312970601CF8BDF8B50C1CD91726
:101A60005F18061C4F40551E092F12D9381C0A2139
:101A7000002B03DA01F01AFF434202E001F016FFE7
:101A8000031C211C2A1C301CFFF7E7FF041C35181F
:101A900013E0002B00DA951E002201E0B45401325D
:101AA000A91A0029FADCEC43E4172C403519002B65
:101AB00003DA2D232B7001340135381C0A2101F083
:101AC00039FF30312970601CF8BD73B5069E041CC7
:101AD0001D1C3009531E00280AD000901A1C201C1F
:101AE0002B1CFFF7F2FF241805E0217001300134B0
:101AF000013A002AF9DC0F231E40092E01D83036A6
:101B000004E0002D01D0373600E057362670013052
:101B100076BDF0B585B0041C0F1C002801D0002153
:101B2000017000256BE0252903D0217001320134BA
:101B300005E05178252904D12170023201340135A4
:101B40005DE0302903D001320292202101E002320F
:101B50000292029E9C4632782D3A50424241B6187B
:101B60000296002205E00A235A438218303AD2B284
:101B700001363078031C303B092BF4D90296AE189D
:101B80006346BE4201D97A1BD2B269280ED006D86C
:101B900063282CD0642809D058283ED119E0752834
:101BA0000AD078280FD0732837D11AE01E1D201CC8
:101BB0001B68FFF752FF04E01E1D201C1B68FFF787
:101BC00028FF331C17E01E1D1B68201C00930023F8
:101BD00004E01E1D1B68201C00930123FFF775FF06
:101BE000EFE71E1D201C1B68FFF7FDFEE9E71A68E2
:101BF000012022700433029A241801322D18117822
:101C0000BD4201D200298ED10023BD4201D22370F2
:101C100005E0013C2370013D01E001256D4205B066
:101C2000281CF0BD10B50C1C131C6421221CFFF7EE
:101C300070FF10BD00B5031C9BB00A1C01A8191C45
:101C4000FFF7F0FF632800DDFEE701A800F0A6F82B
:101C50001BB000BD0FB407B504A901C90191FFF77E
:101C6000E9FF03B008BC04B018470EB403B503AADB
:101C700002CA0192FFF7D6FF02B008BC03B01847B2
:101C800070B50323041C184205D10D1C041C194215
:101C900001D1934201D3002311E0131C40CD043B3A
:101CA00040C4032BFAD8141FA4080134A400032352
:101CB00009191A400419EEE7CD5CE554013393424B
:101CC000FAD170BD30B50B040D061D430D430B0258
:101CD0001D430323041C93420DD218420BD1131C45
:101CE000043B20C4032BFBD8141FA4080134A40018
:101CF00003231A400419002301E0E1540133934205
:101D0000FBD130BD00B5002300E00133C25C002AE6
:101D1000FBD1181C00BD00B5031C01E001310133EB
:101D20000A781A70002AF9D100BD30B5031C0024CE
:101D300006E01D5D085D281A05D10134002D02D092
:101D40009442F6D1002030BD00B502E00130002BF6
:101D500006D00A78037801319342F7D0981A00E050
:101D6000181C00BD08B5FFF753F90B4BFA21186892
:101D7000890001F0E9FDFFF77FFCFFF787FAFFF725
:101D800045FB96200002FFF787FDFEF757FEFEF7A2
:101D900043FEFFF76DFA08BDC004001010B5041C27
:101DA00002E00134FFF7E6FD20780028F9D110BDEC
:101DB00030B5F8238A01DB0013404A05920E134325
:101DC000F8221202114019430A235943CA108318FA
:101DD0001C1CEB345D782478EA336C401B782402B9
:101DE0001C43835C201C5840072319400841800590
:101DF000800D30BD7047000008B5054B011C9842AE
:101E000001DD044BC1180448EA38FFF7D1FF08BDD3
:101E1000FF17000000F8FFFF6440000008B54018FD
:101E2000511A013101F0F2FD08BD08B5801889187A
:101E30009A1A0132FFF724FF08BD000010B5CB004D
:101E4000591A074B0F22C9180023CC5C14400470A8
:101E5000CC5C0133240944700230072BF5D110BD4E
:101E60006005001010B5CB00591A064BC9180023A5
:101E70004278047812012243CA5401330230072BFE
:101E8000F6D110BD6005001030B5B14B87B0D96EEA
:101E9000B04D4A1E91416A46D175A96A1A1CC806FE
:101EA000400F0138062807D801F0ECFC040C1F1283
:101EB00017191C00022409E05A6E16329200D358FA
:101EC0001C1C15E05B6E16339B00D45800230FE0FA
:101ED0009B6DD46DA3420ADC0AE0022403E00C24CB
:101EE000032305E00D24231C02E00D24EEE70D245E
:101EF0002C6148111F2800D922E16A461732944903
:101F000001F0CAFC2000220028002A002D002F002A
:101F1000380040004400490051005F0067006F0036
:101F2000770085009300A200B400C300D500D30061
:101F3000E300E600E900F100010105010F011101D4
:101F400013011901081C00E08348191C221CFFF72B
:101F500065FFF5E08148F8E70A1C0E3203E07E4891
:101F600009E00A1C1C32081C111C1A1C231C01F05D
:101F7000C5F8E5E07948011C0E391A1C231CFFF74F
:101F800054FFDDE07448011C0E31EEE70A1C1C32E0
:101F9000081C111CF1E70A6E1020002A00D00A204C
:101FA0000A1C0E3206E00A6E1020002A00D00A2019
:101FB0000A1C1C3200946C46173402900194081CD1
:101FC00051E001201070086E1022002844D00A222F
:101FD00042E00A6E1020002A00D00A200A1C0E32AD
:101FE0000EE001201070086E1022002855D00A2241
:101FF00053E00A6E1020002A00D00A200A1C1C326E
:1020000000946C46173402900194081C78E00A6E24
:102010001021002A00D00A21504A6846173001904A
:1020200002910094101C111C1DE00A6E1020002A61
:1020300000D00A20494A00946C46111C17340290C3
:102040001C390194101C0EE0096E01201070102242
:10205000002900D00A2241496846173001900292B7
:102060000094081C002201F053F869E00A6E102069
:10207000002A00D00A20394A00946C46111C1734FB
:1020800002901C390194101C3AE0096E0120107076
:102090001022002900D00A223049684617300190EA
:1020A00002920094081C00222AE0012010700A6E9F
:1020B0001021002A00D00A21284A684617300190D2
:1020C00002910094101C00211AE0009222481CE0AA
:1020D0000092224819E00A6E1020002A00D00A203F
:1020E0000A1C1C3206E00A6E1020002A00D00A20CA
:1020F0000A1C0E3200946C461734029001940020A2
:1021000001F02FF81CE00092081C002104E00D1CD7
:102110001C35081C0092291C1A1C231C01F07CF899
:102120000EE0081C02E00C4800E00C48191C221CC0
:1021300001F08BF804E0081C221C191C01F090F837
:102140006B46DA7D024B07B00120DA6630BDC0462F
:10215000C4040010600C0010D2040010E004001051
:1021600010B506490B1C88331A68141C1E34A400D1
:102170006050013203210A401A6010BDC4040010EF
:10218000054B0320191C88310A68013A02400A6095
:102190001E329200D0587047C4040010F8B5114D9B
:1021A0002C1C8C3420680130FFF726FE0E4B0122D8
:1021B000D8629F6AAB6E061C02409A4210D1830718
:1021C00003D420680230FFF7CBFFFF239B001E40A3
:1021D000B601BF10044B8C35374301222F60DA6003
:1021E0000220F8BDC4040010600C001030B50C4B88
:1021F0000C489A6A031C8C331C68D3059B0E91050E
:1022000000D5403B856E921001210A40AA4204D1BC
:10221000E3188C300360024BD960012030BDC0460A
:10222000600C0010C404001008B5084B5A1CD07F85
:102230009A1CD27F000112021043DA7F0333DB7F46
:1022400010431B031843FFF78BFF08BDC4040010A5
:1022500038B5FFF795FF064903230F22051C5C18CC
:102260001540013325770011072BF7D138BDC04643
:10227000C404001008B5FFF783FF034B01228C3321
:102280001860024BDA6008BDC4040010600C001036
:1022900010B5064CA36E002B06D0FFF771FF044B60
:1022A0008C3401222060DA6010BDC046C4040010E6
:1022B000600C001010B5064CA36E002B06D1FFF782
:1022C0005FFF044B8C3401222060DA6010BDC046F1
:1022D000C4040010600C001008B5124B1B68002BE2
:1022E00000D09847104B5A69002A15DD012A07D102
:1022F000DA69002A04D09A610022DA610A225A615E
:102300005B690322191C91430A1E02D0074A01216E
:10231000D166054A013B5361044B90331A68024B66
:102320005A6208BD8C030010600C0010C404001039
:1023300000B5064B5A69002A07DD9A690F21044B44
:102340001140D97712110133DA7700BD600C00100B
:10235000C4040010044B597F9A7F090112020A43FA
:10236000197F0A435A677047C404001030B50B1C2C
:10237000093B012B0FD8084A00239C18257FC45C19
:10238000A54205D0054B08395A681143596002E04F
:1023900001330E2BF1D130BDC4040010600C0010CD
:1023A00008B508290DD0192913D1427808231A42FB
:1023B00002D00022027002E00F2303700723437053
:1023C00005E000231A1CC25401330E2BFBD1FFF78A
:1023D00049FD08BD1FB50E4B5C6F002802D00F22CF
:1023E000944304435C67FF2C10DC6846211CFFF714
:1023F00025FD6846211CFFF7D3FF054A00236C46E4
:10240000185D9918013308770E2BF8D11FBDC0460F
:10241000C404001030B5124C0F23656F85B09D4386
:1024200005436567082D19D0FF2D17DC6846291C68
:10243000FFF704FD6846291CFFF798FF00231A19CF
:10244000127F69465A5401330E2BF8D16846291C75
:10245000FFF7A6FF6846291CFFF704FD05B030BD55
:10246000C40400101FB50F4C616F082918D0FF2954
:1024700016DC6846FFF7E2FC616F6846FFF776FFFF
:1024800000231A19127F69465A5401330E2BF8D1D2
:10249000616F6846FFF784FF616F6846FFF7E2FCF3
:1024A0001FBDC046C404001010B50D4C631CD87F7E
:1024B000A31CDB7F00011B021843E37F1843E31CCE
:1024C000DB7F1B031843FFF797FC0F23021C1A4006
:1024D00022770211134000126377A07710BDC04627
:1024E000C4040010044B5A6E16329200D258121ACD
:1024F00051424A41DA667047C404001000B5064BE9
:102500005A6E16329200D1580139D150002901DAA1
:102510000D21D15000BDC046C404001000B5064BCB
:102520005A6E16329200D1580131D1500E2901D184
:102530000021D15000BDC046C404001000B5094BB5
:102540005A6E16329200D2580D2A03D11A1C293223
:10255000127805E09A18507F117F0001021C0A438F
:102560005A6500BDC404001010B5084B0F245A6E04
:1025700016329200D1585A6D581814400131047720
:102580000D2902DC5B1812111A7710BDC40400106B
:1025900030B50F4B5A6E596D16329200D2580D2A33
:1025A00007D11C1C29342478F020084020435865AA
:1025B00007E09818447F057F24012C435C650B11CC
:1025C0004377034B9A180F231940117730BDC0464B
:1025D000C404001008B504480022011C1C390D2356
:1025E000FFF723FC08BDC046FC04001008B50448F2
:1025F0000022011C1C310D23FFF717FC08BDC0464B
:10260000E004001008B504480022011C1C310D2311
:1026100000F074FD08BDC046E004001008B5044891
:102620000022011C0E390D23FFF7FFFB08BDC04639
:10263000EE04001008B504480022011C0E310D23E1
:10264000FFF7F3FB08BDC046E004001008B50448DE
:102650000022011C0E310D2300F050FD08BDC046C4
:10266000E00400100C4A0023111C46310B70111CB1
:1026700047310B70111C48310B70111C49310B7024
:10268000111C4A310B70111C4B310B70111C4C3159
:102690004D320B7013707047C404001000B5074A28
:1026A000011C042300208A1804E0D118463109785F
:1026B00040000843013BF8D200BDC046C4040010EE
:1026C00030B5074A00238918012206E0CC18051C02
:1026D00046341540257040100133042BF6D130BD2F
:1026E000C404001038B50020FFF7D8FF084C051CC3
:1026F0000021207FFFF7E4FF25770420FFF7CEFFBE
:102700000421051C607FFFF7DBFF657738BDC046FD
:10271000C404001010B50020FFF7C0FF034C207761
:102720000420FFF7BBFF607710BDC046C404001053
:1027300010B5054C0021207FFFF7C2FF607F042108
:10274000FFF7BEFF10BDC046C404001010B5094C11
:10275000231C8C3318680130FFF74EFB064B021C1C
:10276000D8620F231A4022770211134000126377B8
:10277000A07710BDC4040010600C001010B5094C07
:102780000021201C0D22FFF749FB201C0E300021E8
:102790000D22FFF743FB201C1C3000210D22FFF708
:1027A0003DFB10BDC404001010B50C4B00211A1CD9
:1027B000187F1C7801312043187701330E29F7D197
:1027C000936E002B08D0064B1B690D2B04D1137F91
:1027D000111C29310B70537310BDC046C404001086
:1027E000600C001010B50C4B00211A1C1C7F1878CF
:1027F00001312040187701330E29F7D1936E002B59
:1028000008D0064B1B690D2B04D1137F111C2931F5
:102810000B70537310BDC046C4040010600C001050
:102820007FB500230C4A0D251C1C1118097F0130AF
:102830006E469955C60F8542664176420133111C9A
:1028400030400E2BF1D100236C46185DCA180133BD
:1028500010770E2BF8D17FBDC404001010B5074BC4
:102860005A6E16329200D1585C1801392077D15037
:10287000002901DA0D21D15010BDC046C40400105A
:10288000034A0023111C943198320B601360704787
:10289000C4040010034B012194331A684A401A60A3
:1028A0007047C046C4040010044A002313678C32EA
:1028B0001360034B0122DA607047C046C404001065
:1028C000600C001008B59A4B0F20996A994A8B103A
:1028D00018408911013852560E2800D9C1E000F085
:1028E000D1FF08111A2327C02EC0C037C0C0C03B7B
:1028F0003F00002A00DAB4E08F4B9A1840320023E0
:102900009371A9E0002A00DAABE08B4B01209A1802
:1029100040329071A4E0002A00DAA2E0864B9A18B7
:1029200040329279DA6697E0081CFFF797FF93E050
:10293000002A00DA95E0101CFFF7D4FD8CE0002A95
:1029400000DA8EE07C4B596E16318900CA5083E064
:10295000081CFFF75FFD7FE0081CFFF73BFD7BE0F5
:10296000002A00DA7DE0101CFFF75AFF74E0724B7A
:1029700001209833186073E0FFF7E0FD6CE0FFF78B
:1029800093FF69E0FFF726FE66E0FFF7EDFD63E0E9
:10299000694B00225A665FE0FFF728FE5CE0FFF714
:1029A000F7FD59E0644B0120586659E0FFF72AFE15
:1029B00052E0FFF7CBFE022052E0FFF72FFE4BE084
:1029C000FFF732FC48E0FFF735FE45E0FFF7D6FEA3
:1029D00042E0FFF73DFC3FE0FFF738FE3CE0FFF749
:1029E000A7FC39E0544B00221A6635E0FFF7B2FC31
:1029F00032E0514B0120186632E0FFF741FF2BE037
:102A0000FFF730FD28E0FFF745FF25E0FFF74CFD1D
:102A100022E0FFF78DFE1FE0FFF73AFC1CE0FFF716
:102A2000C3FE19E0FFF776FE16E0FFF743FC13E064
:102A3000FFF7D8FE10E0FFF715FE0DE0FFF74CFCA6
:102A40000AE0FFF75BFD07E0FFF74CFE04E0FFF74D
:102A500065FD01E0FFF70EFC012001E0012040428E
:102A600008BD982BBED03EDC382B9BD01DDC1C2B28
:102A700000D187E70CDC0C2B00D178E702DC002BBF
:102A8000EAD0EBE7162B00D176E7182BE6D176E7F4
:102A9000282B00D17CE702DC262BDFD175E72C2B1D
:102AA00000D179E7362BD9D179E7662B00D18AE7B7
:102AB0000CDC4C2B00D17CE702DC3C2BCED175E743
:102AC000562B00D179E75C2BC8D179E76C2B00D16C
:102AD0007FE702DC682BC1D178E7762B00D17BE75A
:102AE000882BBBD17BE7E62B00D19BE726DCC82BEC
:102AF00000D188E70CDCA82B00D17AE702DC9C2B04
:102B0000ACD173E7B82B00D177E7BC2BA6D177E720
:102B1000D62B00D17DE703DCCC2B00D09EE775E7F8
:102B2000D82B00D178E7DC2B00D097E777E7C046B9
:102B3000600C0010647C0000C4040010F32B00D172
:102B40007CE70EDCEC2B00D172E703DCE82B00D035
:102B500084E76AE7F12B00D16DE7F22B00D07DE727
:102B60007AE7F62B00D16FE703DCF52B00D075E791
:102B700067E7F72B00D16AE7F82B00D06EE769E72B
:102B800038B5184C231C8C331868FFF735F9E26E02
:102B9000154BA2660022E266DA6003229862251CC9
:102BA00010401C1C022809D090420AD0012802D0F3
:102BB000FFF788FE07E0FFF7F1FA04E0FFF764F99A
:102BC00001E0FFF713FB002807DDE368002B04D1C9
:102BD0002B1C8C331A6812181A6090352B681B183E
:102BE0002B6038BDC4040010600C0010034B0122A0
:102BF000DA660F229A775A771A777047C404001062
:102C000010B5054C0549201C00F000FFFFF7EEFF52
:102C10000123636610BDC046C40400109C07000079
:102C200000B5044B00201B680F2B02D1024B4A3326
:102C3000187800BD94000010C404001038B5164B7D
:102C40001A1C98321268002A04D0144B1D68012304
:102C50001D4001E094331D68114CA3689D4202D1D0
:102C60006268002A16D0002D02D1002B0AD111E093
:102C70000C4B1B68002B02D06168281C984700236E
:102C8000636006E0074B1B68002B02D0281C291C40
:102C90009847A56038BDC046C4040010AC030010BE
:102CA000600C0010A403001013B5002300930193DF
:102CB000244B1B68002B02D0684601A99847224983
:102CC000009B0878214A00280CD0002B02D0022358
:102CD000137035E01378013BDBB21370002B2FD15A
:102CE0000B7009E0002B0CD11378002B28D0013B8E
:102CF000DBB21370002B23D1154A1360154A136001
:102D00001EE014490968581A44426041400010709E
:102D100011484469021C002C04D08B4202D10A23C2
:102D200043610DE000290BD10A21516101999361A2
:102D3000D161084A1360064B02221960034B1A70D6
:102D400013BDC04694030010B00300109803001098
:102D5000940C0010900C0010600C001008B5FFF7E8
:102D6000A3FF08BD30B50A4D049C286009480160E6
:102D700009490A60094A1360094B039A1A60094B12
:102D8000094A1C60094B1C60094B1A6030BDC046E3
:102D9000A403001094030010A00300109C03001073
:102DA00090030010940000105D2D0000600C0010D6
:102DB0008C03001008B5084B084A196812688A1A73
:102DC0001A6006D5FA2252001A60054B1A680132C1
:102DD0001A60FFF733FF08BD980000109003001041
:102DE000AC030010F7B50E1C0E21051C019200F07B
:102DF0000DFE1A4B03240C279E420FDD09236B7333
:102E000001232B7328E0301C0A2100F0F3FD301C55
:102E100029550A2100F098FD0134061C002E06D029
:102E2000E30F0022A7425341DBB29342EBD1019A58
:102E3000A31A033B2B70621B2B1C01E0195D597315
:102E4000013BD1180229F9D10F231C1B002301E0FB
:102E5000013C2B55032CFBDCF7BDC046FFC99A3B58
:102E6000F8B5104B01221A700F4B0222041C1A7085
:102E70000E4E0F4D0FE0196891420FD01B682B606A
:102E8000FFF798FFFFF710FF002C04D0013C002C47
:102E900001D13C7005E033682A68024F3978002977
:102EA000E9D1F8BDB0030010980300109C03001096
:102EB000A8030010F7B51C4D9B235B000E1C1B4A9A
:102EC000E95C1B4BAC5CEB5C002902D00F22144088
:102ED00002E08021072449009A225200AF5C154A83
:102EE000CB1AAA5C3435BA1A80277F00791A009170
:102EF00007210C1B013210490194FEF7B6FE002396
:102F00000E4F33704124FF35301CFEF7FBFE2A784C
:102F10006B783018D31A391C221C0134FEF7A5FE39
:102F2000013D462CF0D1F7BDC4040010370100006C
:102F30002F01000035010000747C0000817C00003E
:102F400070B5314B314C1A1C9432126890B0A061AC
:102F5000E161002A17D118280BD1C32909D12C4AC5
:102F600012680F2A05D1181C38300E21162200F0E5
:102F7000B1F8A369182B04D1E369332B01D100F018
:102F800053F8FFF733FE0A231F4D6361214E0123DF
:102F90002B678C35FFF7F4FD002801DAFDF75CF9AB
:102FA0002B68B34203D01C4A934214D104E0FFF7CC
:102FB00045FEFDF78CF80EE0184C2368002B0AD074
:102FC000684608A9FFF776FF2368684608A998476E
:102FD0002B6827332B60124B1A68124B1068196844
:102FE000884205D012681A60FFF7E4FEFFF75CFE26
:102FF000054B1C6F002CCDD1FFF720FE201CFFF7E6
:103000002FFF10B070BDC046C4040010600C00104B
:1030100094000010790D00003E270000A00300106E
:103020009C030010A803001070B5254C00202368F5
:103030001D68FFF715FF23681A689542FCD01E68CB
:10304000FFF7D4FD1F4B0A221F4C5A6118229A61C8
:103050001522DA61231C903300221A60FFF7C6FDA7
:103060002D3601232367FF36154C184D0AE0FFF774
:1030700087FD23682A681968914203D01B682B607A
:10308000FFF798FE23681B689E42F0D10E4C182073
:10309000231C903300211D68FFF752FF0C4B281CA6
:1030A000196800F051FC3834011C0422201CFFF781
:1030B00099FE044B18229A610022281CDA6170BD27
:1030C0009C030010600C0010C4040010A803001042
:1030D00090030010F0B501240DE005780B1C25408D
:1030E00006E0C65CED0077083D43C554351C25401D
:1030F000013BF6D5013A002AEFDCF0BD30B504E023
:10310000845C8D5C85548C5401329A42F8DD30BD6C
:10311000F7B5099D0AAC2678089F2C7894461D1CAB
:10312000002A0DD118E063465B5D4A5DD218131981
:1031300001920024B34201DB9B1B0124435501355E
:10314000BD42F0DD0AE0CA5C12190024B24201DB84
:10315000921B0124C2540133BB42F4DD099B1C7055
:10316000F7BDF7B5099E0AAC2778089D347800288A
:103170002FD000292AD01E1C9446002A0ED1013FD0
:1031800018E063469B5D8A5DD21A131B00240192EE
:10319000A34201DADB19012483550136AE42F0DD8A
:1031A00037E0CA5C121B0024561C01D13A1C0124D2
:1031B000C2540133AB42F4DD2BE0D15C49420C1B1D
:1031C000211E01D0E1190124C1540133AB42F4DDC9
:1031D0001FE000291BD0181C002A06D10EE00E5C4F
:1031E000135C0130F31A1C1BE40FA842F7DD10E05A
:1031F000CA5C0133141B013462425441AB42F7DD17
:1032000007E0D15C013349420C1B611E8C41AB428B
:10321000F7DD099A1470F7BD70B5049D01242C7078
:10322000141C002905D10BE0065D0A5D96420BD106
:1032300001349C42F8DD05E0815C002904D10132B3
:103240009A42F9DD00232B7070BD00B503E04318EE
:103250005B78435401319142F9DB0023435400BDB4
:1032600000B504E08318013B1B788354013A8A427D
:10327000F8DC0023835400BDF0B5114B1A785B785D
:10328000825C1A4000D040220E4C0F49231C261CA1
:1032900004C32C3600221A6001240A1C123117784C
:1032A0005578C75D3D4202D01F6827431F60023238
:1032B00064008A42F3D10433B342EBD10020F0BD65
:1032C00091010010280E0010DD00001030B512230F
:1032D0004B43334A0131D3188A0051181A785C786D
:1032E000825C144204D02F4A5F24521894705470A8
:1032F0009A78DC78825C144204D02A4A7C245218E2
:10330000533214701A795C79825C144204D0254AD5
:103310007C245218A33214709A79DC79825C1442AE
:1033200007D0204C5F226418251CA235A1342A70D6
:1033300022701A7A5C7A825C144204D0194A7C2486
:103340005218A03214709A7ADC7A825C144204D04B
:10335000144A7C245218503214701A7B5C7B825CB5
:10336000144207D00F4C5F226418251C523551348B
:103370002A7022709A7BDC7B825C144204D0094A5A
:103380002E245218A43214701A7C5B7C825C134287
:1033900004D0044B5918F43127230B70002030BDA2
:1033A000DD000010980C0010F8B52D4C071C00250E
:1033B000201C20214F22FEF785FC002D04D0221C6A
:1033C0007C23393223701370231C4F3300210135C5
:1033D00019705034052DEBD1214B2D22181C38309B
:1033E0000270181C37300270A1209A705A70400089
:1033F0005F221A541B481A54A320400019541A493A
:1034000008784978385C014204D0191C5331523392
:103410000A701A700024211C381C0134FFF756FF73
:103420000A2CF8D1114D124E00242B786A78FB5CDF
:103430001A4201D0315905E03059FEF763FC0D49BD
:10344000091A0A310C48043400F0EAFA0235242C37
:10345000EBD10A49084800F0E3FA0520F8BDC04660
:10346000980C001041010000910100109C00001018
:10347000B000001093010010D80D0010897C0000EE
:10348000F0B585B001900027FDF7C6FA6A4C3E1CE6
:103490006A4A7542754113687D19002B00D1D5E049
:1034A000002303AA537023687F210B405C2B00D1BB
:1034B0009EE02BDC382B00D192E013DC072B6CD084
:1034C00006DC022B00D19BE0062B00D0BEE043E0DF
:1034D000212B00D188E0232B00D18FE01C2B00D0C2
:1034E000B4E089E04F2B4ED007DC3F2B64D0402B5B
:1034F00064D0392B00D0A9E066E0542B00D17DE0E8
:103500005B2B3ED0502B00D0A0E06FE0732B69D036
:1035100010DC662B39D005DC5E2B57D0622B00D037
:1035200094E067E06F2B3CD0712B53D06D2B00D013
:103530008CE02CE0792B4BD007DC762B4ED0772B10
:103540003ED0742B00D081E046E07D2B23D07F2B32
:1035500025D07C2B7AD135E031231370022E51DD3A
:10356000231C083B1A687F231A40542A07D0032ED5
:1035700048D0221C0C3A12681340542B42D14C22E2
:1035800006E032233DE033233BE0342339E03522AB
:1035900003AB1A7036E0362333E0372331E03823AB
:1035A0002FE039231370062E2CDD231F1B684722C2
:1035B0001940232926D1EBE7302322E02D2320E0F8
:1035C00041231EE04222E3E74322E1E7442318E0DF
:1035D000452316E0462314E04822D9E7482310E0AB
:1035E0004C230EE050230CE052230AE05222CFE796
:1035F0004F2306E0552304E05522C9E74E2300E09F
:10360000492313700E4B03A8291C0022FDF7F8FA7A
:1036100023681A0605D5E91D0A480022084BFDF764
:10362000EFFA2368DA0572D5E91D07480022044B3A
:10363000FDF7E6FA6BE0C046280E0010A00100106E
:1036400000000010F53F0000917C0000236801227B
:10365000134206D0A818C0B2002107220223FDF7AA
:1036600059FA23680222134205D0A81DC0B20021D6
:103670000623FDF74FFA236804210B4205D0A81D4D
:10368000C0B202220623FDF745FA236808210B4247
:1036900005D0681CC0B207220223FDF73BFA23685D
:1036A000DA0606D5681CC0B2042102220623FDF703
:1036B00031FA23689A0606D5681CC0B2002102229E
:1036C0000623FDF727FA23685A0606D5681CC0B200
:1036D000042107220223FDF71DFA23681A0607D5E5
:1036E000281C09300222C0B20821131CFDF712FA6F
:1036F0002368DA050BD5EDB2281C0930C0B20B21C6
:103700000A35FDF7F1F9E8B20A21FDF7EDF90136C6
:1037100004340C370B2E00D0BAE6114B1B68002B7B
:1037200005D01048002109220F4BFDF769FA0F4D13
:103730000F4E104F0024019A2B78D35C6A781A42FE
:1037400006D0A3009859E15D0922074BFDF758FA0E
:1037500001340235092CEED1FDF768F905B0F0BD52
:10376000CC010010937C00000C0000109C000010A5
:10377000A4010010D400001038B5FFF751FA00285A
:1037800014D006240321201C00F0DEF80321C5B26A
:10379000201C00F02FF9281CC9B2FDF7A5F9092C4F
:1037A00001D10B24EEE701340E2CEBDDFDF73EF9E1
:1037B00038BD000070B5041CFFF75EFD201CFFF74C
:1037C0005FFE0A4B1B78002B0ED0201CFFF7ECFD90
:1037D000074CC8235B00074EE518211C301C5034F1
:1037E000FEF738FAAC42F8D170BDC046B103001004
:1037F000980C00104E3B000000B589B000280ED098
:10380000FDF7D5F801A80921FEF718FB684612302C
:103810000A21FEF713FB01A8FFF7CCFF08E0FDF734
:10382000CEF8044B1B78002B02D00348FEF712FAA7
:1038300009B000BDB1030010957C000000B5FEE7A3
:1038400000B5FEE708B50A4B0A4A0B4903E01078B9
:103850000132187001338B42F9D3084B084900221A
:1038600001E01A7001338B42FBD3FCF76FFEFEE7D9
:1038700000000010EE7C0000C8010010C80100101C
:10388000540E001002B4714649084900095C490011
:103890008E4402BC7047C04603B4714649084000DC
:1038A0004900095A49008E4403BC7047002934D0AE
:1038B0000123002210B488422CD301242407A14202
:1038C00004D2814202D209011B01F8E7E400A142BF
:1038D00004D2814202D249005B00F8E7884201D35A
:1038E000401A1A434C08A04202D3001B5C08224332
:1038F0008C08A04202D3001B9C082243CC08A042A3
:1039000002D3001BDC082243002803D01B0901D08E
:103910000909E3E7101C10BC7047002801D0002003
:10392000C04307B4024802A14018029003BDC0463C
:10393000D90000000029F0D003B5FFF7B9FF0EBC95
:103940004243891A1847C046002941D010B4041CCC
:103950004C40A44601230022002900D549420028FA
:1039600000D5404288422CD301242407A14204D22E
:10397000814202D209011B01F8E7E400A14204D20E
:10398000814202D249005B00F8E7884201D3401A25
:103990001A434C08A04202D3001B5C0822438C0847
:1039A000A04202D3001B9C082243CC08A04202D3B1
:1039B000001BDC082243002803D01B0901D00909A1
:1039C000E3E7101C6446002C00D5404210BC704751
:1039D000002806D003DB0020C043400801E080201F
:1039E000000607B4024802A14018029003BDC04679
:1039F000190000000029EBD003B5FFF7A7FF0EBCAC
:103A00004243891A1847C0467047C04600B500298E
:103A100005D000230139037001300029FAD100BD1F
:103A2000F8B5041CA30719D1231C04CB0F4D104E6D
:103A300050199043021C201C32420FD1181C0B4F0E
:103A400004CBD5199543354208D1181C074F04CB38
:103A5000D51995433542F1D000E001300378002BB1
:103A6000FBD1FEF758F9201CF8BDC046FFFEFEFE54
:103A7000808080802578000D0A413A200020202592
:103A8000633A20000D0A4D3A20002020473A2025B5
:103A90003032780D0A0025732025730D0A00444D3D
:103AA00031355F530053455249414C20434F4E53EB
:103AB0004F4C45007265616479000D0A4279652EAC
:103AC0002E2E0D0A002573202573202025694D48D0
:103AD0005A0056313400202025692E25303369568E
:103AE000004C43443A25303269202D20256900508E
:103AF0005245535320454E54455220544F20534174
:103B00005645007475726E6564206F6E00424154B4
:103B10003A2025696D560D0A00444D3135000D0AD5
:103B20002530327820200057616974696E672066FD
:103B30006F7220646174612E2E2E0D0A0042616442
:103B4000206D6F64656C0D0A0052656164202573F9
:103B50000D0A004F4B004641494C4544006F6666D4
:103B6000004C43442064656275672025730D0A008C
:103B7000000000005C000C000C7C287C7C447C2451
:103B80001048285408000C00384400443800201025
:103B9000081038108040001010100040002010085D
:103BA000384438007C006454484454281C107C4C31
:103BB000542438542004740C2854280854380050D5
:103BC0000080500010284428282844281004540855
:103BD000384C5C7814787C54283844447C44387CD5
:103BE00054447C14043844347C107C007C00204015
:103BF0003C7C106C7C40407C087C7C047C7C447C5D
:103C00007C14083844787C1468485424047C047C70
:103C1000407C3C403C7C207C6C106C1C601C6454E0
:103C20004C7C4400081020447C00080408808080FC
:103C30000408007844780004040200007F010905AC
:103C40000000070000000000070B064400FF0144CD
:103C5000004400FF01440B0600008C001201FF032A
:103C60002201C40D0782004500250092004801444E
:103C700001820C060000E60019012601C0002001A7
:103C8000070400000000010002080400000000FE1C
:103C90000101020804000000000102FE010B060001
:103CA000008800500020005000880B060000200013
:103CB0002000F80020002006030000000400020B92
:103CC0000600002000200020002000200603000045
:103CD0000000000109050000800160001800060BCB
:103CE000060000FE00010101010101FE08040000C0
:103CF00002000200FF010C060000820141012101C7
:103D000011010E010B0600008200010111011101D9
:103D1000EE0B060000600058004600FF01400B0655
:103D200000009F00090109010901F10B060000FED6
:103D300000110111011101E20B0600000100C10197
:103D400031000D00030B060000EE001101110111FE
:103D500001EE0B0600008E00110111011101FE0899
:103D600004000000008C018C010804000000000029
:103D70000208010A05000020005000880004010B21
:103D8000060000500050005000500050090500008F
:103D9000040188005000200B0600000200010061B1
:103DA0000111000E0D077800860132014902390227
:103DB00042027C0E07800170004C0043004C0070F2
:103DC0000080010B060000FF01110111011101EE3D
:103DD0000B06FE000101010101010101820B06FF3A
:103DE0000101010101010182007C0C060000FF01BC
:103DF00011011101110101010B060000FF01110069
:103E000011001100010C06FE0001010101110191D8
:103E100000F2010C06FF011000100010001000FF5E
:103E2000010804000000000000FF010704C00000BA
:103E3000010001FF0E070000FF01180024004200EE
:103E4000810000010C060000FF01000100010001DB
:103E500000010E07FF010C003000C00030000C0014
:103E6000FF010C06FF01060018002000C000FF0142
:103E70000B06FE000101010101010101FE0B06FF1D
:103E80000111001100110011000E0C06FE000101CD
:103E9000010141018101FE020C06FF011100110028
:103EA00011002900C6010B0600008E00110111014E
:103EB0001101E20B06000001000100FF01010001F9
:103EC0000B06FF000001000100010001FF0D0703C8
:103ED000001C006000800160001C00030D071F0033
:103EE000600080017C00800160001F0E0783014498
:103EF00000280010002800440083010D070300047F
:103F0000000800F00108000400030E0781014101D0
:103F10002101110109010501030100070008000A40
:103F20000100181110133831303378717073C8C123
:103F3000C0C38881808384848782C5C4C7C27574E6
:103F4000777235343732151417120207020802014E
:103F500000030109030402040205030500062024EE
:103F6000282C383C4044484C4669726D7761726534
:103F70002025735F5631340D0A00252D3130732012
:103F800025732573000D0A5479706520273C636FF3
:103F90006D6D616E643E203F2720666F72207061F8
:103FA00072616D730D0A00557074696D6520257519
:103FB000730D0A003F0025730D0A0D0A00564F5974
:103FC00041474552203E3E200025630048656C7005
:103FD000004E6F20706172616D73004B65792070C7
:103FE00072657373003C6B6579313E203C6B65797B
:103FF000323E202E2E2E0044756D70206D656D6F43
:104000007279006C004C6F6164206D656D6F727920
:10401000007400546F67676C6520646973706C612D
:1040200079206F757470757420746F20636F6E7370
:104030006F6C650062005265616420626174746532
:10404000727920766F6C74616765000000800150A2
:104050000080025000800350FC3F0150FC3F0250A2
:10406000FC3F0350EAB820226077373A812A339424
:10407000CFF87C5798A0396BFCF718377F727EBE5B
:10408000AC0F12A47073761C0C817246B11A35D233
:104090007022707C0D6E3C2154F4FAD5EF09B513F3
:1040A000D698FF88360AB8E98A7B197E279230664F
:1040B000871181362D00882542BA65DA4D93BCF907
:1040C00087C900E7720FBCF17B7530EC72B27204E5
:1040D000D1796C11FC24E88D5D48719E680C2F3EEF
:1040E000805D5508C121C9F10CDBCB1700BDB0D7ED
:1040F000049ACF060BE482CFCA6E46445D404D92CF
:104100005EA4D2AD14F3AE437B67EB32A10F57E947
:10411000306DD7637AF2F236A2D11D7B200622CC15
:10412000FE6910607B7445C8FD8DF27985BA4BD26B
:104130008DCD43E4235B0CA07398106E8556849755
:104140001F5D4DBE3ADCAC903A2670BE4DD5AB2417
:104150009881AE730FB84C2E10E18E98EB0E843A16
:104160008C4C49A3B9C53E5417CE9FFD145C310B4E
:10417000F4184C31304204F20433FAB146A61D3E25
:10418000BC798D90F845CECA549F594CDC4A1EDF4D
:1041900041CA20590A457777AB4DA6DC58853806C9
:1041A000B121EDC18B1C0C6347E225038FBEA295A4
:1041B0002938816A21F77B98514899705FED64AB8B
:1041C000C489887CAF5692E9738E01E6688564DF06
:1041D00033FDD82B134ABD8955FBF1CEDABCC9FF9C
:1041E00096FF27960462E3F673F462841EA97BA50A
:1041F0005ECEE20FE483E32F50AC21B7583AF76864
:1042000077BC43C5DA9A215109558BBC3896613188
:104210005CC4BD6D3273DF3AB3085E38712203CBE4
:104220008C8BA7A012E2A454B5A54AEE4EAF3BB9C1
:1042300030FFDAA8C948D73D2A4F14847AFE96C8C1
:104240003E42E61DCF18A02A3C349C480985B3F5B0
:10425000F5C53EC1866D5D432591B139D9522873AC
:104260000DEEC5B673A2B71FA4FCB67A35B8F1F748
:1042700004EB9BF3821250DEDF2AB5240454C07C89
:10428000274628989BFBD40A25B5BCB08F42A624AC
:104290003C913EB885A7C5B66A873BED8F40EDA936
:1042A000FD94405CEBF8D5ECC331B157CFAC7594BD
:1042B0009FD93F8E00D8D925844BD8094E71239AB7
:1042C0003D3545CEC346A74CE959AD26C6463457C1
:1042D000BFBA936A990AA748B1A263FEFC84179DEE
:1042E0008E3F4985008E09FC6BD0CD6DE9A8E5CAEB
:1042F0009C7A1C66077351B0ADAB19F5087BC34BB4
:10430000D81A467F5DAB620AF6C0889836F4A06979
:10431000E31A1925548EC423D6D788C39EA70D0F40
:10432000C71FCF912E37411FB2FB9F8F6697F402B4
:10433000D1EA309A90700885B6BB61020F8692B3BD
:104340003B157367D70BC178D7E9F824E0FD7B668E
:104350005B3E0CFCA76F125EF116EF1AA83DB2DFB0
:10436000242E496EA5A0F16F30F8222818599F6EAF
:104370004873C4AB8F9E7AAF7423B44529E8C6490D
:1043800035FBE2AC559D8293D3898FB6962EC0A89B
:10439000B452CBE2119563C1210EDAF48CBE11A3A5
:1043A0001C14F54FBF23EA8781EEF7E5C21A01CD51
:1043B0009C028519727CD68AF363C962161E515B12
:1043C00047F3525E7498AE048A3CA74C0B8F293891
:1043D000B06F7F28C9F6B1EFC5FA27BBAD3FCB5F01
:1043E00065E4CA7B97A51E3CC0D22D42634F39E9D4
:1043F0008317B6F0E9929CDF988DC71A2DF71483C6
:10440000B153048398131FA173BFD4593FF138727D
:104410001D2651F5AD8FDE747C19E9BEB82AD16C2A
:1044200007663749E54366B092E90B3DE53E8A51A0
:104430000CF0DCFF9DD6E9CFB7FE9E920EFABE5F70
:10444000D653FFD2091EC0A7513A0A2ED45E0F6B75
:10445000CEF711087D7524698DE8C7EFBECB59C929
:1044600083C4D50CE7B8660857FFF9CBB19C0BBEE7
:104470008A504B0B2A37A9F8B0142191F2871A19E8
:1044800010D119DD7AB6D5A3E23B49CEAF298EE82B
:104490001B8209DEF6C2DE3CFBBF9602A3832231FB
:1044A000A36A700FD9AEE6925ED1B48EC95C747FF8
:1044B000BADC7DF5AA74F3A7CF641182B1210E2A6C
:1044C000E25043B825BBAD2CD32FB874168ACB6607
:1044D0005A350724B7B7E64E3FD9789EEF9654BFBA
:1044E000CADBB3BD4585B6146F47B153D8D4175A4C
:1044F000E4F95E777407F24AD8B2073249E1ACFBBF
:10450000423B9C01BBF2809CEB1A8EFEFCF15F9F4C
:104510006D631C1B0B3D953F8AB13E98DC4CFB97AD
:104520009D494D99EE503649E2A396CAA61E5938C8
:1045300096AB20BA671893A4F850C6F7B2866F8777
:10454000A570A895C72732F33D53A82A4D0BED1F40
:1045500036E2EE0025947D7341CE06CEB4CA384BC8
:1045600012FA386E9D40947194F96712F5B91CAF38
:1045700092B6CAF7D3DBDC3947B92DA98EC9D2036D
:104580008720BBEB933877C522F0A76AAB54C66986
:104590001D365E3114D168B59575CCCF2920B28C0B
:1045A0002F4F2C36091A088531251343C930FF0DCA
:1045B0005CBF485543C9210D4BB385454302D17AB1
:1045C000904B2DBAE0EB259752C30A9791DB58C563
:1045D000DA24DFD7B3407C6AAF28E396FAE5663485
:1045E00070A85E3207F6C1191770CA15C5C1B8C5E3
:1045F00060AF0A24A610AD1E554CA0DB57F318DEA1
:10460000E63300230CE5DF5FC30B8D056CB38861D7
:104610007D78C3450D8F937B4D4AAF01218AFE9D66
:10462000DF8456E884F7463C8F90955275CAB8608F
:10463000CE783E5389D974252CAB718058C52DF0A6
:1046400021AF2628AEA88E65D759B317664F1A56E4
:104650003C72B2DA1EF3D07841CEA1C8719A1F0520
:10466000AC7DE6AF01174CBAF98F4781E2BBF78A00
:1046700075E4EF526313325A37A9164FFBA716A2FF
:10468000EA0EDEE4CC39A100A7A659BC77C60A7EA3
:10469000F1B683184243710FB813D4CF8A59272734
:1046A000996EA5BFC5C8273498E6340980D7A76797
:1046B0006E0E41B53B8CD6FD94B5DE4DF99112825C
:1046C000655B03EC6213E9833CD560D2EDBC997E57
:1046D000E38414006EE3C9F143468B2179CBA294A5
:1046E000B9B2B588725E06163FCE83BBBB1A2F994E
:1046F000E46C41089E18B88FBC52F108F8A299BE2C
:10470000A8FF143C32CF2BA099D1BF957C2CF6BFCB
:104710006A210A939441C2A279E9CA4EAF158BCDA2
:10472000E4E5A4CAF070210BFD60CAEDBEE19BCCAC
:10473000D2DF3557822BEA217CA900FE32081B39D3
:1047400023B9D48F6FE7DF5F4F0B893C4387367BFC
:104750008736A009145753E296F84FF12891555126
:1047600036570FBD1143AF3BACB0D850673A26BAAD
:104770006D9AB8337F4CF8F6C9FD9E4CD17564171D
:1047800091343C0A07DEEABE2606D56BF22F4802BA
:104790009C66396501A483C49CBE9E7CC2CD2F1645
:1047A000237FCDFD62637CC8189627121E8A7B5337
:1047B000E586F5D701C258B65995E8DB864A6CF014
:1047C000584197276AD91C46B26C43411987577ADA
:1047D0001A2CD010691B83F4172A445FC2825B94A1
:1047E000C86F3843D500B3E32B1E0CBDBD7C5754B6
:1047F0009E22C055DB5765BB3A1D18AA0BF5A51ABA
:10480000EAA4D5CDC79D53F8B22CE4CF2D25BA67C5
:10481000218EF6D50A1FFAF15844D5034E86BA6F99
:10482000131ABBADA36B09B6E2369DD73ACBDFA412
:10483000B39E78F3C73822B181A224A4ABBE5B3308
:1048400091EFE8A4EDE34F6C1AA773F656DB54A67C
:10485000AB35125268517476E6036CE52B7D6D5FC3
:10486000705619FC9FBBF0540EA3DA97CB85044A0F
:10487000FE8697C7D353CAAE11416DE13EC20A709E
:1048800019A20CECBEFE70D8AB8A37D5CDCFE3C3EE
:10489000CECA27C507B19E8A084B155DF9B17CF0D9
:1048A00059A80C11BEE16EF38D16583F4AF16058BD
:1048B0001D0B79C883B7B59762C3316033D07D577C
:1048C0009F85FA12E587B34F779B07EFBA106B9776
:1048D0000BE1B8EC3029DCDE1055A6E30C19738F20
:1048E000A38E5FD1966D0746B148A2158CAB96ABEF
:1048F00050CAF31C6545568582832B9FE287280C9E
:104900007E61984017F35BF457E930A18B1E222E8D
:10491000E9F506CA59797ABAD4F7FDE668F8E0E411
:104920001935011822A5CB882573B1165FFD8B3A86
:1049300009A85D14400D15CADFCA9B3621D37C63DC
:10494000735417E6BDF3D3D58CCB5B468813F3DBEA
:1049500091D243C6CC6EF91DE6C68DFF7B27F88445
:1049600002ECF44FCFEF5F05069845598AE69D2289
:10497000B3115271074C304364D8EAAA3C7661C047
:10498000548EBD172BCC30B0B0C03A7E45B9C2D3DF
:1049900062D2CD1619B55900515919586C9E11E3C0
:1049A00027DE6E8E3163C6CBB9A27BC502F8F47FD9
:1049B000FBF49443C7C9C82EE13871A353A98E559F
:1049C0003FFE26ADBEFF8A11098BA07FA880F04C68
:1049D0007482FC6B429286CE811796EB348003770B
:1049E0001EB4CBD4E8B27ECB14ED515C3822F0D8A3
:1049F000772C360C70959B86852B9F8CFEC8671D87
:104A000061126D72E6DD282EF01C2F47A85D056F40
:104A100038F524735105810EC73E47C44BA126C00B
:104A200079F44A0683577A9F1A5238F84F771DD186
:104A30009BC8B4CB5A77F6E95D888E8FB82A3F7150
:104A40006AFDE99F8DDF1A8211018DACB0AFC10AFA
:104A500051EDED0A2637CA209E0EBD9830DE128633
:104A600003C160D8BA643C74FDD5CC81EE25F3BC9B
:104A700038278BA16B037551DE2BF94D42F69A6CEA
:104A8000EF2F332B18657B8489252F015E7FECEF98
:104A90008871396073E752C8368F3655F883CEE295
:104AA000B5AC03F655E7FB7836CC75C5C62FA02C00
:104AB0002DD170A5FDE5EAB83763ECADF74519D205
:104AC000BEBBC32BA27D83094F4B1F35E0C89BBFE4
:104AD00074EC48663A62CCCC5B44472F3C98FE1F8E
:104AE00003FF3C1CDC9272489A540D877B6949D6BF
:104AF000845E302938138BD98664EFB1847C07AB90
:104B0000812C733B37DE2A21F3CC0D464E4AF54EFD
:104B10003FA61331673B45A03E49704C2B69536B50
:104B2000A66C2116EE4E5030E1C0A8F7EF3E0F1FE5
:104B3000E626F9198DBCD0980AAA74EF5D28A6095B
:104B400013A87B9F47F55AC38798ED418252ABFC6F
:104B5000B104BCFCB123285D2D8FD02798AD48C38C
:104B6000E11E069B99A8CA4E96002F968CAA762520
:104B7000F197EF652092C601762D383059A267D59E
:104B800087722E8E7C16F662BEABF599A729F2CC01
:104B90005B14376656C7FAC3A47A83699321F2EC93
:104BA00052580D4B7C3BE9AB110ABDBBC4EC9210D3
:104BB000910168FA9C63D610ECCC59264F65E22728
:104BC0006445B03542A515A7E66B07B3F55C1C59E3
:104BD0009CB874E50188278ED8C1AD0C00EA72B28A
:104BE000B6712951C32A96A8A8BADDEFF1A689E0CB
:104BF000C2C28BD190E47C4AB9C2B5CBA3F3BDCB82
:104C0000434FDCF1B00E29D6702B6F4F33B4D70170
:104C1000745F398FC8478024E2D28627DFD964ECDD
:104C20008A28EE6D3C74FF2967059020AF8F54E50C
:104C300054B3789245DD2A532FF3BF3152B8197E11
:104C400093BFA98AED23C23976BA9C2EC514B268E7
:104C5000FF0CD446C47D02BBC6564A875D76185DFC
:104C6000CACDF25FC2FCB5589EA404E33BB57D1DDE
:104C7000E409FFABC389EDEEB2244E6935A71CD918
:104C8000874D4B7AA4CB5F1A70FBB4B9CDFE73038A
:104C9000114E572383B384694A9F9961FFFFEA5AF3
:104CA000470FE5DFD5E74C9DDE4586C13FFDAA7A7B
:104CB000A5123EB0612FFBA665DF87377A459111BB
:104CC00069CBE821A83F2FCA40B975DD4D44EF3AC2
:104CD0003A9842F0EC4D1B4D9996A95689D4E6A11D
:104CE000F28A94EAAB7F7100BA136CC668898B951F
:104CF0002B575B8DD62C63783173B966C103C1BF66
:104D00004222E46FE4990EC39E0E8F6490CF5D76CD
:104D1000B1976B547027E16B9D196762E8504FCED5
:104D2000232FCFF5AF931E54B2FFA9BD49047C21B8
:104D3000B23723B3B296079073263F0847C6F48C68
:104D4000E4F15D182ED26B71ED30E78790F43311EA
:104D500033378EE560B4874F8CBBE13901095116BA
:104D6000C366D6680AA44FA5ADDB05CD7B9B6EC29A
:104D7000530A457C956A778DFF944A42B0A9144640
:104D8000D281F69A51A7FD118D6A86CF2FDB375F4E
:104D90008D11DE7517833D2136424112342912E10F
:104DA0004BC97904C18271F64A93B3C7656CAA3EB8
:104DB0006543B12BF2D37B12FA329BB03F5083C6CE
:104DC00098C3573EA8D2FB0F32A534B21037AF3785
:104DD00049B1BE316D663AAFC70333EB4AEC9EEF83
:104DE0006642037A513DFE10FA848323F7E3ECED2B
:104DF000898234F23E6531D5749535CFBCB073BD30
:104E0000CF43FD1C231AB3A24F4E9A21EE84AD83EB
:104E1000636606FE6EF50B03F88694A1C13915D8BA
:104E20007FB011A4AD0C83CADE3009316C54B712C7
:104E300069364B490A075AFE236138FA8471EF76C6
:104E4000A7038E60273CA9B3F87BC938AA6B9833B7
:104E50005CE9291701DE755AACAA7F4689B7746CE4
:104E6000DB313904FFCE0A1A9845F083469127FFBB
:104E700004F11143CE5FED6BF62FBC3F6845AFB335
:104E8000A01226EA85FC7A1A31618252509BE0F02A
:104E900077E2396F8245765C77BE7BCCBF1EB15915
:104EA000E2E30A005062C22A321490E06F6AC9A39A
:104EB00032214C793E65E8DBAB4197A5109E7AC75D
:104EC000029C7813C66E1D3DF1A172FAFE3A0BBD2D
:104ED000701BC9BF6221C9C9BCAD80F16F4B27E40B
:104EE0001112E40DFAE0F04FAB215E1B1CBC8155A2
:104EF0004C692F58C421AE9041C552A7C41C6AE525
:104F0000A78B5E29F6280CF3206F1150A12F864441
:104F10003B210A3807B16EDE6F0EC3D6CF1454178B
:104F20009732D6FD836B9B73FC360106A5C05FEDFF
:104F3000307144E2067178B706539F150393CCABEA
:104F40007B536C617B6E97B725CADC9D2DDAA8A2D6
:104F5000E44A88AF102376F50108FEB781D5D5B1B4
:104F6000A98BC86BED458895DDA363D6C778036828
:104F70002E45682F3A50919F70E8BA23A761738835
:104F8000BA4F6B677D71328EC0D87BFA337352A7EC
:104F90009A7C8601FE5D16BE07EF4F3AACB93D76AE
:104FA000292588C1B5E18D94EF24621FBA900DF5D3
:104FB000E77D08A52C00782747BBB219D42874C90F
:104FC0000BC0AD0F446F7BE1AB99111FB2F3E06DE5
:104FD000CC03BB8C9E83DD42E5ED4DAEE378C4741B
:104FE000D009D1C756B7843C8BE38042F8F6881FBE
:104FF000A0A3BBF7107E191F4F40756D3CE30D60F9
:10500000D6AF405AB294241E78ABBA3177A505507A
:105010002A63401EE044EF607085FCEA6D3D2AB0D3
:1050200044BBB0126BD47F95F5AAF0460AE57773BE
:10503000931BC50990839DF6F3B445E6B82C1A334B
:10504000836A818AD5EBEE0958FAB7ABDA7D9BC546
:1050500030D2E02C1DA40EF07218EF21C8773C224C
:10506000898D5CED5FE52861D1D4BA181E818F6A05
:10507000B91CDBA87BFFAB6F89622DC5B6F0FC4C79
:105080007E27B396492AF2DD1DB4FBCC6FDBE69197
:1050900025A42A08DD3D8094896D070A0821D7F5EB
:1050A000C280FBFC2393068371074B01B63D022EA1
:1050B000FF2A4131B1DDC33FB805C8088B2706B5CB
:1050C000DFDD75AD7BEFA008C210D8D1D78B54FAC5
:1050D000DA9083B3B36EF946CA7FB16F0B351A6DA0
:1050E000F7435FCD5E6F9156C59C10BF71E02BD426
:1050F0001C2644D524AB4CA58232306FB3CEA64CCF
:105100000F6A42CB504D7D3ABF8A9B28F35C7349AE
:105110004BD2E646F44F239BE7B12A96C3339196D0
:10512000B46F673706E618E8511BAC47551AB983C8
:10513000C5F3ED76FE37BEA59610F3E132386B9CD1
:10514000B6737EA7A2AD094F78C027EDF5B043A78F
:1051500037D7FAA488DEBD2A8D0271165474D53F64
:10516000AF9B5922887B0F6E642E6EDF165548E385
:105170001871AD56F1E496D1F68D9DE42AC9D72E6B
:105180008CC5664600D221201F078FADF2F8F4F5DA
:105190006C0245F10595EFA82135DF479127A19CC9
:1051A0002176163D85A99D2700583217793D8974CF
:1051B000B2FC5248751BA5B3E0F0C9C72BD7B7277F
:1051C000C7A546F0E4AB4B31DE21A61A662D547C10
:1051D00056078A38C7F965383EB25C46725337CDF8
:1051E00076F188D3AD5F404F947403A57B0C56577E
:1051F0006528AF065A8CEFB09E2DAFF57AD66C6954
:10520000E18D77DDE507F84FE294B59B29A704FF10
:105210003811281AA749008BDBADD05765A3293E6A
:10522000F69C94DFF89128B9E9B71621A16AA6ADDA
:1052300091487241B9DDEB3B39A916F15ACC042DE6
:105240003BE167514976556755AFED9F2F7291F657
:10525000944405434A7D3D635EEF3F85DD16F96169
:105260002BC17662CC421651ACAD9DFDC38903982B
:10527000928929BCE6552733D8A3022A44798DD6D2
:10528000417826C3A6CA112DCE2C79461771146A0F
:10529000013232C4410981D32F84F0F4EEEEE8D715
:1052A000A0B4CEB07B4368C8C725A19B1D50DE6962
:1052B00047F0FDA2BF15D3F2B552D1CAB8EBE1EB6E
:1052C000E9821D06A7EC5A82B0723DBE5146CE9EC1
:1052D000FAED95BBCF117E2A9AF7A7ACB71671E409
:1052E000AEFA4B0F253876D7701AAFA1019BFE237B
:1052F000D60BE8D9B5A6461D1DFBAB1A183B0ECE42
:105300008947FB4C9BCC2D675B0372A4A0F43859F2
:10531000F74A9101F487995A6AABD36FF483459D9C
:1053200003B135319A721A5445CD1081D290F5F7F8
:10533000DF605B8D939D4933C97E76EB8C543E8B49
:105340003F47A2ADFC14E3411DE42BC17F3666BD8F
:105350001FEAA84D8CED922A41380BC5996E81AE9B
:105360006F42BB79F4C2C1CB0F8F76DBE66FED9154
:105370002AA97AAB32EA57C59AE6720CD4C171FEFB
:10538000651DCDB7971AEBC44E275935A4AAC08323
:10539000E14D9DC902110E6C4C4B71F0ACA91F92EE
:1053A000250BF4B39B278ADF350017A1A9C6ADC62C
:1053B0005CAA1FCD14187157436D9CDF8E3134B039
:1053C000C4ADB68D1F8DD906BD39A5965CDD238988
:1053D00014525B839C63D67347825CC31C18C78AD4
:1053E000E8A56789AF24AF85CB3A8F47D7A8587116
:1053F00093776B02CCB6A1641A5974F79340F0C945
:1054000029AA5C15C8C5E489CDB6E9C6033D6F324B
:10541000A2030F68F637379416D843D050C1DD6D1C
:105420004F14FBF22646E3989E07B66B8E83F4C4B6
:10543000194461A744FF5BE5F53F08EAAE4CBE2C7A
:105440006B3B9D2851C5C97EE8C12AEEEFA61874B2
:10545000BC726DCD2F03270DCB46C9B699A987A97C
:105460006CC010E617ED71FA61521DBDCAC1E1E0D2
:105470005B7BEF19E10465A09EAF9E5E99D5FB565C
:105480009A7F4426C60D24536CA22CBC1A3194A3D7
:10549000039FCD5AFFAB082478E9161627488FAD35
:1054A0008C258A45F243CFD5E4BA88F9D35D630CE5
:1054B000E16B0BA0E1369ACC6FA82FD3CEA8EA9966
:1054C0003DEEFAACC4A6760AC9B3A2B4233A55633A
:1054D0003F5500496AC99C0E0D949744209A27B203
:1054E000C5858350F098ADE0F04DEE7CBED323C36C
:1054F000BF01F5B4B6767BDCE771EC536ECA5F355D
:105500006BE991CDB330F44FDC55B77EFF8450F892
:10551000DC5B99FD0E858891F8A5EE5355973D17F4
:1055200098ECA106366736AFEDAD81326B4690F050
:105530009D32DC7093EEFA679AA3AB699DAF0CD4F1
:10554000DFB009D2B248EB6AA207309476E824A310
:1055500011BFB9C6911EAFCF86992B966C0297DE0C
:10556000CE183F0152B209FE3ACFD25670153DE631
:10557000B3CA9B1BCF44E69FA46E6EB98EC29689B8
:105580003C6A7CF800C387E84A2553B953BDF6C787
:105590003134923BF3DAE35356D071630B73E91065
:1055A00088CAFCCB8FE84DB676D97D0F7FCBC4DAA5
:1055B000991C3137487CA72110A7C94E67D524B95B
:1055C00034F5D9E3A4C6307A80B2CCAF25C8FB8DC0
:1055D000F986E64B2AB16FB7761BAB11ABE58EE9C6
:1055E000382C02F5BF43230A7A9F057310CC34167A
:1055F000CEEEDE55AE877D975E3552D8042AEFBEDB
:10560000EC3385A1D7E5562071EFD8394595148D37
:10561000F757D38F6087E2C29FF0543AEC7D92FB3C
:10562000EEBF9BF2AD451D3FCED79CCC1D1C393340
:10563000A5D2851D5E0837C912C0EE8778E135D244
:105640006F0B423B8FEE888CAC72BADBFE17688A18
:10565000EB2C3D911DC9777144DEC3D4DC35ABE141
:10566000CBE9824898877962A74F6D4C7BC051B3D4
:1056700092A64EC91081BACE6B333FDA63595EA150
:10568000D3EA21D95E211E8D2D1A444956C00BF351
:1056900051C6F7C221AFFBDCB274995E8C94660CE4
:1056A000179E03B4714A63F26501F7CCED193474A7
:1056B000560A5B81AD89DDCC458DD8AC60C925B576
:1056C0007FE7545A2A1FFB5D05EA1FC25B4E3E105E
:1056D0002B325E05560B724D13E5257516C075A16C
:1056E0004FF476CDD63B833891079A5612E62D5D5E
:1056F000F9E67DE76166ED2B6DFFFA5AE72118E6C2
:10570000E8CDE41ABFBF3B79A1F74FD29D69B63807
:10571000456FEA2A0FCD4461599C1D9CC8DD7B660C
:105720009F24E310DEF79B261E3A5F8A8BF798C80A
:1057300006ECBC242A337C0C9D264B4C9E58B3E1CE
:1057400059D756C05BDD181FEBA109FC86314CED23
:10575000A94029C0AE9C6A04D3BE1FCB5D45D0844E
:10576000AADE89F317FDC7192F62D45260DB571EDA
:105770002E6C08001B21A44B36218B5C4180549376
:10578000D95A2B67A22E0A02956F27D5F6BAD138BF
:10579000DE44FF1BBBDDF7EE2736E50CDFC18DE8ED
:1057A000B3523BDF83D3C669D3B9EE8ADCC2238E02
:1057B000E80D83B39210B2E10A24DF0EAECEFD866F
:1057C0007EBDE670761B7E817D59497A59DBD528EE
:1057D000435CB19BB4FEBDEDA8945FD64391BD4C34
:1057E000008C78918AD86F99B6A5E8D4B09EA906A6
:1057F0003C695218D15392728639FC0233B204E8E4
:1058000093B159BDDE9198E5AAB29B1259F70AE807
:10581000A01E3B20310390B6B81B5C1C9CB2697D76
:10582000148C883831E4F19C494D5534587F95E10A
:10583000A62A096F81376E3B32AFAB651D11A6FCFE
:10584000BEAE4B07CFB4EE91EB05CCF82BEF09EFD2
:10585000B309696AF2135D9A561A9A23B087002633
:10586000EAABC026E404B90B694B659F0345C472DB
:10587000C80B8645227E3939EE2591A6D16D634449
:1058800012D0D2D048BC5E597EABB65F775F3B6327
:10589000C738FDC86089F7A4E2D7710C7565595304
:1058A00051B11BE5CF70026EA9006938DDB5E5A3E3
:1058B0004E705BC332F6D41BFEDA732790396F0E3D
:1058C000056E29871F3EA11E9674743FEE8AE4C0C0
:1058D000039143D6603D1BBD8747346C08463A3080
:1058E000B83338303E1665268701DAAFA68D3D9570
:1058F00096354EC31650E9CFCEEBCAA28342D20BE7
:105900009C0ECF942707EC334F8E12D98CCB3AF1F3
:10591000132C4ED13095DF62E398A6A894064F5B16
:10592000CE3ECA61238E0C47D8BDBBBF7CBC773648
:105930007E9ED0BFC8423A04B2668F19D05396718A
:10594000C54A56DBF78BAC645502257D86D8A1D8B5
:1059500011B24ED136D34044EAAAE889E45111305D
:10596000013CFD2BD50E33A3A104663554CBBE6696
:10597000B6DCD1F5890EB167A322C7E533CE406C02
:10598000778FDCEDAF81CB05FB9B2DE8BB25CD7D73
:1059900012FE7D0BCC389F42CE234D6B3B920AD931
:1059A000E4220B4F6858E9385D6C39AE1B46149EF3
:1059B000181C986E841520FF540DA171ED1F00BEB8
:1059C000B42F9C38BC848BCFE972B1366F8A56FDF8
:1059D000E065E975D8EB6AE3DFE2A91640361DD130
:1059E000FADFFE28CBB5FC4113BE1112F754EC01CF
:1059F000E4C366947C21FD0B4223458C2AC30240FC
:105A0000EEA4EFFE5D819A3864F7FE851E7305B43F
:105A1000EDD3FB61C992DE5F2F777CBFE44936E3AB
:105A2000BF8D5C45DEA0DDB555759680E6DBF606DC
:105A300003B4EC22B3AF7F3EE03402A2ACB75B32DA
:105A400028291AAD27D3D4AA9223672F5EC85702FC
:105A5000AF13A00E3A1E5A9879C882BD63AC6F840A
:105A6000196CF5F6C800AB51CE2C7E8EE8DEDB4219
:105A70007E7C2FA8A9ABD887883812F0B3EEC52951
:105A8000E94F25108E627B928BAD051EFAFA69777D
:105A900049D978F66AE877D605F6970C39D997E5AB
:105AA00010FE47F5F1DCAE1F0E7BBA5C14CB87BC51
:105AB00084710AE609049062B8BDE970DDD4DA4A5F
:105AC000B20F4B3E298F4F60865B46D8002ACA141E
:105AD000EF012BFA243509B6D900CB8DBF5CF594C4
:105AE000C5FA37EC5D80A28B088780A096037D7194
:105AF000663DE8E4FB42D93A1B18C152664EAF68D6
:105B000006CBFC0E97507658D8A2BB94587B368BA8
:105B10007B62CECE77EF87CC56C17F12C3C6E29FA1
:105B2000FB5F054580A2F3E01E869D9167ACC6D55C
:105B3000CA93B7393834B2085246C962C19629C6E9
:105B4000E3FCCF67C2BD52AB7F01E28673B126BBD7
:105B5000A895C76BC6CCFDD1356FBA49AB4E6780EF
:105B60003A92260044D1A3584448CF406B138F6625
:105B70003FD28B6CF81A926B2BAF4FA56C38694FE4
:105B8000096F7462EC10B8FBB98220AB20C16D04C0
:105B9000172D86F28164158CCB84D8103813170C1E
:105BA0004B7ADE9B630B598CD47053017FD54A69C5
:105BB000C74B08E3271CF88CCAA49136A45EF813DF
:105BC0008D47B2EB6C6FB1E5F8B212CCC50E430451
:105BD000A5FEB000FBF0C6357C654E0D18F1B59AF8
:105BE000B93D8891CF936F5D84B5823EC1BB433F81
:105BF000B6DB9B791479E66058DB765C9AA88D64F5
:105C0000D2BDBC7A1B489BDA9397454F80A580E6AE
:105C1000BB2C72B7E0F2D7C094ECEEDCEFD2260BCF
:105C2000CC6193C19A9C4C962A0EE5474D63DE6584
:105C300092A07E77CC3E20F189FBA8740D9B8867EB
:105C400053FECDB282280D0DA9DF389FB1EE3B6A1D
:105C5000BB49AEF32E4E7B8394A706D2CD54E927E1
:105C60009D66E86DDBAB4480E94A86EA1B82784397
:105C700027CF50163B55A1C2A70018EE955692BCEF
:105C80002EED7D97A270FF023C4766FB4388AC90E7
:105C9000210D5D38234C4296A483CE8EB2B99CDC94
:105CA000CD5B20D721CB56CEBA3B8747FCA8ADEAC7
:105CB000A2A5EC0E917349E6A280F642C08560DB96
:105CC000B844FF7E20366869A004F75D4E14544B3B
:105CD0008C2D868261DE767F75728F3F2B527243E8
:105CE00006A4AA18DFB5D4EBAA24D6BCABA58CA910
:105CF00017C93DB3A3F7D9351ACFAB2C45F7E2E767
:105D00009361950D19D7A0362F2CA2B7D103FD436F
:105D10008BAEEA293A5B0E02541EFC1A737C56D0F5
:105D200040F69AAF851E19C13A27B3C7CFD4622374
:105D30000A277E7E00CBD7E1A383B34C9A15D46E9D
:105D4000DDAA08949756944456078966B4F6D3267C
:105D5000DD086D3DC5EDE280794DA8D4A0741843EF
:105D6000DF334C9E4BFE14B5822632109B8B081EEF
:105D70003F0932D32693C180877B9A8FC00385C1A8
:105D80008223FCCBBEE67637328CCE461498992B14
:105D9000DC8D6AD20C432B388FE5B1A5A63A8F2152
:105DA000888793A1EC538025A57635D8468925555B
:105DB0000F194E1A99A3889973E1DCAD6086920B96
:105DC000CF1E6556C1D795D3590DFE4E20539C0D5D
:105DD000BB44B178975D25BE6CD614EC710D4B14A5
:105DE0006D2E9C214BAA954BD3689361B7EFD99444
:105DF000B076AB6A1F642F39F9AE9CBE507EC25399
:105E0000700BB00A9301137DE1F11087328C6D1293
:105E1000D9253CF0C32D5193D200B297FCE3A17178
:105E200063A3D3B083881E03B23FD4CBC48A2E446D
:105E3000474A903D47B3BD584F09C9085BDB24A9C9
:105E400079CE590FBC3C8B94FE093ECF745B402D3C
:105E5000C75567A0610C7B0F6ED131483EC0075D0E
:105E6000A46089834622B541667F80C12D919353FA
:105E7000F23F1208CE441D849F26ED8E767440D3E7
:105E80002C28BA6234A9D060EFC485B4912DFC35BA
:105E9000E4591D29A3CE00687D257CA18CC9A88A60
:105EA000ABA1B0CE76290E060D48219C7AE0D6EF44
:105EB0000C68EC267BABE56292659E83F566175D08
:105EC000A7A70FFBFDB7C11E9190F16CEE9D6BAFC4
:105ED000114CEB68825E9BF35D784C710D5A1D6D21
:105EE000061A79E118A9B045C6D754F6F68690BFD0
:105EF000C9DE04E1DE8F13667D3E8C3378725C8DE3
:105F00009F01C5BCF2B3AA82DD6F43A1E9A0E2FF05
:105F1000ABC760BF48CBC0724BB54542B2D566E84F
:105F2000E59BF65E0E84C44BD46B60FC718A5936D7
:105F3000EDE4EE48069BE9BAC95E10158720176D9F
:105F40002BAB885572B01F04539937C0EB2D050455
:105F5000C3062CBF6BF5C895B132D7DA578E5244C1
:105F60004C89A356595F24BC04B33958C65281AA40
:105F7000D470A3F4140F2E919D93E0A1CC89C1C2DB
:105F80008A816FF7F49A281D73B28F09724C6926C3
:105F90002894CF795F929B9CD5E1087E11672ACB2C
:105FA00077709D4A255517054F1D57A700D88D13AB
:105FB0004D963E15806CE6B2EFC89D48C96EDA4E2C
:105FC000D88F509F8DB51D2ADCC6202BF9F199F78B
:105FD0000ED5F213DEE5B886113CE226FF02CE6153
:105FE0001DFF7F0B108340F66F919B92259BE79BD3
:105FF00023CA5744F983EB9EF2E1DF222B87052A5F
:1060000050BB86F5299094C9321B57DC2E2E88810F
:10601000CC69946B31F0962A9B94FE1C675A84805D
:10602000F91C59CC11D277C29A4281A5E9D21D063A
:10603000F71ED787395C08CA4F57D620C8C3A40DAE
:10604000CDF19F8E40EF92E29A494F889D7D19F3E2
:10605000A0F8BE9ABE5482E9A6CA026482CC149EFD
:1060600047F028A8A1207CA8760BC6DAFFCF351B05
:106070003B704A76852F2F7B373EE66C69AF4882AE
:106080001E5FDEB8B67CD26E0DDB45005F5136B3C5
:10609000897725D518A741DAA25319813309ADE9CB
:1060A0007AB5CDF06D5AF6620E8ED38B06219575BA
:1060B0001E3A947EFAE6F64D91470FFCFED077EF3C
:1060C000622261AC63636FE20E622182EEC913AF9C
:1060D0007836ADA08B419D796D9C0D2A312380B01F
:1060E0002B1AE9CEE0E30902AAD06ABACE7BA960F6
:1060F000964D8CD02D1D220DCF3599C187377660F6
:10610000119C9531FB583102758BD4CB462CF5D8B8
:10611000BD6CB2828B6A5926FD023D222F847649DE
:106120008DAC6407B28E08C8CB69892B34014D321F
:10613000D3820A620C9D2138FA52E6EAB0B855BC07
:10614000D901A087607155C63A0E45F4B4422122A8
:1061500038E0573C44C3D6FECF18165E466C01B5F6
:106160009993F63A617CC1AC29241F2EBE3FAD6CD9
:10617000926ECCE26C7019C72C9AE909E5CEFB034C
:106180008153BDEF78803240A3D75A7787C7B8E6EE
:10619000F6EAB102CB8A42ADE4B50C20EA8EC8B76C
:1061A000AE422DBFE453615C0FACEEBDF2186E0938
:1061B000967F02B2B10B40D91D2621B6994CDB2542
:1061C0001818E888D384A1618ADE376A410109C1C1
:1061D000EB65E0862ACEDB2DAEE5564F8BC0A5A938
:1061E000B9EA3F2E1D15BA14F6C092949AD1C4593B
:1061F00075BA8F15E54EF99C051314D3BF03C9C2B8
:106200007F826541B7BB87BD67BD6B29668685A761
:10621000AC28EB194813D4EE2ED1DEC30D5C0F0071
:1062200053B0E47B97EAB1BC7B3621AACFEFE49070
:10623000B54E959FB534FE5C58A0A7477E747C226E
:10624000D7EED09C0321CFA11A1153985222B30844
:106250000C28CBC39196E2B425EFD12E28337B9E38
:10626000A9F39A9BF9B7DF1AFF0D254B7997A51D66
:10627000AA9B2A94DAF3DBFE841BBB1AB32076EECA
:10628000CBB5D83D34B1F69E88F3AC4642377CC6D8
:106290000620BFAC2F31FA942A24387CBE84B50284
:1062A0004ED59ACFEDB0D7ECD4A20956E84950C7E5
:1062B0000FF168D4CDC4A16B00ED0115980419FE4F
:1062C000966CA4FBF7BE2983DF2999FB0D02951D6F
:1062D0006AF04C4DD110D28D5D7BE78EF55CD54CCC
:1062E000FDBEBB65DBCBD97A79B27E5D83D3759772
:1062F000099A27AFCD39F6BE0184D6964D9F532F0C
:10630000A9576CC5B0E1FBB9A8BE5DF163035FFAA4
:10631000E9885C3CA9BED3E6C4ABB184DE1330008F
:106320003014CB2493595D6442A65AED9C148FF12E
:10633000A91904A0611BCB602B0B31CF4EF08DD679
:1063400023B8BFE4182AC0D1A0B011A30A09940849
:10635000E3BAF882663B8B675B0D5242B89EF583C9
:106360009999A335CA12326895133A15F71EBCD114
:10637000459FABDA4FC6CA1C62B69423BE24B6341E
:10638000FE8484302EFD27052FC0C795B193CCBB6A
:10639000C7C3546C88FF419C5BC323B0F3D6C9D4F8
:1063A000110BC6C5392D7888BAE8F7368DF9CB06BA
:1063B00070EFF033194738049B9DAA420E31A47543
:1063C000C0C4E0433310601F35F7FF7693289ADA94
:1063D000874DB5B27FD71A93A19AB4159B9D053E00
:1063E000EAB6DB2F5A43E99F5224016FACCEBB3F84
:1063F000FE1A54BFEA0C755FC7ED79501F04FFB851
:10640000FE974790DC1E8B5858BD4805FB06137954
:10641000DC6C60FB7BAC1622CB30F8A217E02DDBE6
:10642000CF70388FD5510F133EF40D4011F879A677
:10643000C19DDC3FCBB854F14FB08AC300D3165A8C
:10644000CB87151D7A02B8DFFFD78502FD5CDBEA3A
:10645000EBAAB4EB78C572169E595153A07BC323A7
:106460001BE482F6E4AEA93832B6718018EA6CE417
:106470003D6391321725A2B20BC746809856485407
:10648000182D435739E6B5224257784B82C33D2237
:10649000D0B18EE9F0A72C756C9F920DD5333621C3
:1064A000E30C06A6D7B78A626C00C1658FF3701043
:1064B0002157A6F2C7D7BC695EFAD145CB39C7547C
:1064C000922C5B8CB711D721753D57BDEC57DBCDB6
:1064D000B0BDCA688BCE5C90B978D68BC5ED999467
:1064E000149C854505F4FF93FE4DE163C4CF8DA157
:1064F000FBF3BA51C4B4192D3CF908907AE9A2E033
:106500008D3EE8B0B8561683CDBC477867D13E0AB9
:10651000D71529A45DC6F6A0E0676C8390571AAB27
:106520008AC1337009829132FD8AE7232D9E791248
:10653000240B747CD1BAC798D12FEFD876DE6DFDCD
:10654000B32D1F1A00922229203AF874E3D7609ADB
:106550002C70ABC56786D3EE24D42FF9B8118324F1
:10656000E6C055EB82839FE64C5A35D570F7FFECB9
:10657000899F6055C65A26D7BB81B9092C6CAB7F61
:1065800002758D0F4580E667D9DBF0EC208CB19E5B
:106590000B0D281F68F10CE47EAC459DAED0A6D74C
:1065A0002D5B7F6B21A5DA7B4F6C132414924B017A
:1065B000F30385B952B2C8A7E92EA0BD56529A5727
:1065C000679275664F268B1D49FB8511BE1435D524
:1065D00085331389E75BE8CCC9ACD9E93A4FD810C9
:1065E000D91913DB129198823AD17FDEA9C23046C5
:1065F00097401B347F2C14C7B6B34D34532CDF00A7
:10660000BE97A8646DBDFFC6F2A8B4C126D24EC81D
:1066100012FCDECBEDB7455B78D60933347E95AFFF
:106620009259139AB620B5CC74ED5BD82CE7DAD426
:10663000DECEAE11DFCD61C17016EC6199E75CC2B0
:106640004BF2461DAA75BB33CA6420C81923029CAD
:1066500098F684DCD3D12C7F0FEC829F2E79245EB8
:106660002269378F3258C46DA9F06B8DB48B5F905F
:10667000DAC7D74A146999CEFBBD967DEA27EB129B
:10668000602B7E5482119EF6F0BAC49034B9B0B536
:106690005B33DCE4E3261BD1C339375B845873B129
:1066A00080B9A10E62087FCA83B36292F9B24869C9
:1066B00094F3D25E2A5886B7E9BB8736F056B33FCB
:1066C00085EE939427D54AC1E33B7DA1601915ACB3
:1066D00003BB32D1F26AFC8942E217EE343AF7A8E2
:1066E00042C795F23730AD29B1C04C56BC28296F4E
:1066F000FED67A98B748306C480627FC39B86F91B7
:1067000067957FA28BE63A9F9E6BB719E791B20916
:10671000F5ECF06E4C96A4EFDDF8703EA31A1C5118
:1067200011D9411642F11BEF7E3A3F4D04317355AA
:10673000B9FBCCE898DA1042ECE419729726F153D1
:1067400067264B61D2AF2909141D1F69FBB5E6D03E
:10675000FFD33992AF8B0CB0DB22B32FD69B0D0742
:10676000E9F61AF928ED4AA098127C5B9F736AF744
:10677000DC37FBBACA71E6ADD678E821D1CE67A284
:106780000E8EE7F042DECC0702450BB13D191A9898
:1067900056E907914496DDF9BB0F8EF3F12EE652D0
:1067A0009A5912D9253F0DA0D8FF4ED644D62DC9EF
:1067B000D461E9366D786AC50CBCE9FBD9FEBECA66
:1067C000136748E24F173D3E0F24C640DDEA6E389E
:1067D0002C2193484C479438336F6FF504965381BE
:1067E00073047914A4C156DD06A558952A2B6DAC07
:1067F00080517509907FA791D35F22E2A96C4B2845
:10680000350E8A48CF7EA79F5456B954553846CC8A
:106810002C7B4E3AF1B50F3A2D64897AD4CA108E8A
:10682000C3250FD521B3140FFDABEC2ED49FD07E22
:106830003D2B9851FF6737F166D9C1D39172299EDC
:10684000280E1BE00634BE788203CD8EFBE2B193A6
:10685000EE8899D634A5F5F173D02446D7BA56ED13
:10686000766FDD78E6611006625C84E6AD405926FD
:10687000C9D4ECB658DE1B85EAEA6B64591FA470D4
:10688000DB450B4341F89748D4D199C5D4514034E6
:10689000277C2CBE046EAA44FFD103D9E9D728086F
:1068A0000C27CE89E2EC42F283C589EC230472B155
:1068B00014FEC22E9A038BFEA6B361413943F2BE89
:1068C000E679108F3CFAA3ADF590E2905AF2832E50
:1068D000D8F61FE5D888A55BD71F88B66965706FA5
:1068E000B9B7319D37F28E7807A28B7E6EC9C55736
:1068F00047A410DA78BA69D016CC2EB72EAA4C85E8
:10690000F608A972EB3B97CF88C02B438AC31D4181
:10691000A205D6513AA0D79148E772E1D2BF4CE721
:10692000AEC8CA35CFBC45DCE9473CA0CB68003FC8
:10693000B45E3828A3E6C3E3207CE3B098074A5E40
:106940008C51179CF9F6B77C47C58A4D898EEE515C
:10695000F8C4474B64A5BE6EFA6012BCFC61EE073A
:106960001816A94A1884D397C22BDBE348ADDA3C4A
:10697000A447D9E781F7DFA1DA3C23E49037E24B63
:10698000E4D5808001FBC143298C23AA8BCFE9C1C8
:1069900052125274BAA09825DCF647760B2632C5FF
:1069A00072C5A5872F01F0472AEFA9190E9BD76161
:1069B000C2ACB99EDB54955FF43596F2207D416AF6
:1069C0003472C75F483D18DFC9BCB438D9D9D1DDAE
:1069D00094A083C7C01A452957D0EA008008D71B66
:1069E000C9EADF0698A0B6D60D3A1082C2DD4AC0C9
:1069F000D80D9934F3026D8D63E34A63766F5CB012
:106A0000E59878694A22E348E2CBEF408F8FD77050
:106A100068D3476BB03DF2C3E33F3006A9B9F1EB51
:106A2000EF72215DC599A0A64ADA051F2D98BD48D1
:106A3000BAFFA8D5C635552ED041718977CAF9E37A
:106A40008F5AF8DF73FC1965EA9BEB7737D772979B
:106A5000D244200D5D4CD886AA1A66F0F2BFFCFD28
:106A600076887B5F26CB4F5106C8F7CA243873F06F
:106A7000FBE7FD0AADE9C5F5FD5DDAFCB0E0FDB070
:106A8000DABDDF7D4380D14E3479C9E5673A06C768
:106A90001F850323096903BC96D74AC499C8589433
:106AA000315EB8137C328D87AFCA56629191F0DCAB
:106AB00069B4953858722B1FD1BF11F8CDAB2E1B7E
:106AC0007B27C642E84E6EEA96D1EBCD3B0D1C1FEC
:106AD00033CF0C84395D28811E9BA48E4012D4C410
:106AE000F4B5E2DEA4E2B942FE4CAB58631776601F
:106AF0002379D6CDD68008756D51AAE2C86551C8F4
:106B0000FEE8BFCCE215A25982E4086389E55EF68F
:106B10004EDE5E564EA20AA154D86D4FA8C41A2F5D
:106B2000155E5C759673298A7CCA69433854890757
:106B3000C2AE738D2594305A748D3BE28190E38D03
:106B4000E1417646D11E785CA67E79DBA6659C285D
:106B5000D8440A4C3A400D5E237AF8F81556AFED4A
:106B6000F200FFCCDDEC6161727FD7317B3109F03F
:106B70000AC5F6C8412EBD22681919F48DB1F32F4C
:106B80002EBD05C2AAD79C595FE8A99CBBD49FD152
:106B9000E983E38C27623E72CBAC64B8BE7E60B3FF
:106BA000248771CC1357D40DC315DD7F76560EE1C3
:106BB000E0AA62D0AF989FCDCE888C94EC1402747A
:106BC000B918391B2C5F23D7D0EA123C005F5E2432
:106BD000614BFFB45748699E187EBA104677B0F0F3
:106BE000B38C6D16DADDFF03DDD05E5E91EA78D7F7
:106BF0000752A35FBBD630632E9B91D576C63CE38C
:106C0000EBD8B4DA66402D65D9EC18F0B8B41B3077
:106C10008D127B19C0FB809570EB24B7127839C8B0
:106C2000EB5113F067638821F033F8558E41CB5F49
:106C300097A670AA2AC02D7EB738D97E057923A4DD
:106C40001A999F1A2E9469106E5FF09EC22D39C258
:106C50006F21CAA44B3EDF09D84B84CBF7196E02D3
:106C600085BBCF59FF6EB6226392687C7C5215C4F7
:106C700020D948CF9D65BCD567B7284AEFC0AB4E39
:106C8000DC4887383B38B419DAA2B92F48004B26C4
:106C900012011BB41FF55956A2E5CA25CEB47FF5E3
:106CA00081E003CA062761B4C0B9AF1E9D1B689777
:106CB00038CFBFE131A6D7FB9520278B4B6050EA38
:106CC000A89C8B3D76E9411AB796538C8B29E985B0
:106CD0001279EDCB2E8181C922C4055B6423C81AC9
:106CE000BFF92FA8A161609D6C8C6E80FA68444B3F
:106CF0003DE53978F7E014F0BDD363749A4BD5F5D0
:106D0000119CB4F3C12F23ABAFDB177B7376D9C5CE
:106D1000B1B5F0F48CF88E40DA590F4AF5AC66EC58
:106D200046B267F66D30CF5134B4DC114DD3C15447
:106D3000448CD2B31094CDC369AD88CF24AA5A62D3
:106D4000CCBCDD48C0B34288FCAF3A729B9CBC7798
:106D500012521D5965661E149FC566C024074FF266
:106D6000C615D0DF48B0E4F1CD3891E40879BCC253
:106D7000511C9642CA8F4D970536E1C31398A7144C
:106D8000CE6D7AA026A1D7922DFABF2FA40A442D4A
:106D90004F10186BBB0D39BB6C53C179AF7036887F
:106DA000D9723E5049D312E4D7B348C3EBAB9597A1
:106DB0002C7B94F8F3D00B0F1C4E9ED8E0AD662DC3
:106DC0003C7F12A2BF948B073808747D9D6E881497
:106DD00064219C7E6C27CB181624B8F3776F114E74
:106DE000AFA589D6E7DB6A538560897252FDC50578
:106DF0005B879EC93FB56B74730435AF90600558CF
:106E00005448BCC14669142874CEDC794C41E9D899
:106E1000CB82FE67E774F1BACCD53B4FD5E9E07978
:106E200043F860160B4CB5440A6DE663B2D8F275B0
:106E300058C8FCBEA83586BC7DF4ACFB6D4A5A44EC
:106E400035D4FBAA924E146B088B7695AA27B4D63C
:106E50007E93EB1CDDC4CADC02D1FDF8862619A1A5
:106E600010164678594086B30324AEE97B1C572E92
:106E70007048913A041ECB32C424F1E1890E2B579D
:106E80006CDA999D827E3354DE58DFC0DA1B02EF44
:106E9000D3CDE7B26612F4C84EBD5241773CF90437
:106EA00030C0A157525BEA4C609755EE056519CD8D
:106EB000360674D238F3022DB59759A295D81CC85E
:106EC00005EDCE1DB97831C1D1CA36E62D66A5D102
:106ED0007B13F5F38E5CBCB7979ED3F79EA897986B
:106EE000CF04DDD0F717A09883C7AAD25D42190955
:106EF0008E6AC1E5BC0A41C0D0EE39C374BDF11839
:106F00001B6AFC599320FB757C6D476BB010B28DEA
:106F1000BCBCFAAF2FD40FFEB0455C0F41696E6068
:106F2000626494FC68FD42AA198E31194E3BBF621F
:106F30001A620418700D77452F69DFA1DF9DB4A692
:106F4000D36C3CAB9D38849B26B22802957F82DAB5
:106F50006777C1B706767112DB8E02899D86FDDBED
:106F60009874D59F3318AE7EE95E6722450DA06EFA
:106F7000050AD0859BA1C6BAD0404A6907A0E29B0A
:106F80000CB46E3D795B85C4B045BE1CA5DC83E0C6
:106F900091284FF9550A0644E177AF4F7EF0066815
:106FA000070A524B628C975721EFB06C7E0794977B
:106FB00026E86D4A19500CC84534EB2869308D110C
:106FC00053499119D8E7924A961C515A7F32589EDC
:106FD00059BAE5DBFC8A2C87A929B0304C3747B178
:106FE0002AB4D1E965C87610DA6407AED9564050A4
:106FF00073F63DB97D0597332F1DBE6FF2C197E53E
:10700000B64668845EB510999CBD56B344EDA6E8BB
:107010007561891C76045B8D6E651A9CB2A7FE842F
:1070200035095F1B890FF76C35B13DB0BEBB055EFE
:1070300004928C9866329D7EF4F8EDDF5B981C37E5
:1070400076ACCEADCE4C6482F828C574E207D2BDD2
:107050006067196CA7C153B7F9AF87705663B4372F
:107060004FF7694B4E44494060D01561BEEFEDF4D7
:10707000E01D255197460D1523791DEA5BDF746FDE
:10708000AD22645C7F327FF99E7B4B0AEC6C58D555
:107090007347BD5A93DE7F8808CF47B8E8763E1F16
:1070A000F1DA1CF9CAA2529BE2F19D41F971FA573B
:1070B0001B0A2A8CD2E1FB91B8B0770D01D0386160
:1070C000681FEA23638C3D0C46294AF711E22B44E2
:1070D0006EC4CF0E179C55FC47EA9AF09B90E2498C
:1070E0009A20210106AD4FEA06FC52C27B7AEEF5EA
:1070F0006DC03A85822BDD8B3F00FF92A1DD4745B5
:10710000EDC3AEE7D18933B50C967FF15F1A024C1F
:107110007AEDFAC6664AFEF08918808AB01A513CA8
:107120001D14BE57BDE2BA161A0184C448EC98CFAC
:107130006E039503B5BB5F1D1E7D64F40A143E8289
:107140006EA6E02A0B7ACAA5C4F878E36F0F694EE1
:10715000597EC2824000BC2F7F7773B3DDBAFCA991
:10716000A9D5477C34BB28494358A96F77FA7E38A4
:10717000FE561B7B9B0EE3EF56C68B912D4FCC45E5
:1071800046750C1314D34FFFBAF3735A2D3071E0C8
:10719000EFD846018FF5C257A8BA8B53231E506F04
:1071A00044FFCE76741D3473BBEAD36287F75BBBB2
:1071B000934426BDF45B516DA046F25F0B05EFC60C
:1071C000CC344EEACAC298EEBCF3F76F2B9D782DF3
:1071D00046F98949BD7C45E67BEFEAD555A9228E63
:1071E000D31863603A90AF3DE84A7EF83C5FCA54DA
:1071F0003C38C77414EC67FA56174AD1FE51E5D3F0
:107200001EEB4CEF48B03B51D981850C32C584F15F
:10721000EA191301944282CCB1B35662BB0D2B1A0A
:107220001B9C73615C978F3F3C1ACC27A624EA9085
:10723000064A26FE14734436AA4758869E27024AF9
:107240005317DB91629E681BBD238550D54EBC222F
:107250004D51D1E41470292AB232E229DBF3C67011
:107260008EE177C65F3CCD09732B02B82F65BB2139
:107270008C73AB3F03D9E5DDB788BF15231E0F48DC
:107280004C142DCBE06F0A94D381C0EC07BBB954EA
:1072900060348FCA35486984383070E8FEB5F14BE8
:1072A000309DFCD07BA3B16BD709509D87F1E1D213
:1072B000808A59EB3B5EB9BC685CF5592B918165BE
:1072C00075E7E75ECC52824B9EA717146D4ACB98A8
:1072D000A8113492E89976F1BA9C098F1B7C40F989
:1072E00050061A045F8B62898942C45B147D75EE77
:1072F0007BD1904577E761053534E4B02878753265
:1073000098A21EA6B4C776C03BB6A35E9087250E92
:107310006A3B72CABC24C075236136FDAB152FA72A
:10732000F518631E958BB78F434D5E339919A4539F
:10733000B8A2FAE3885FD761D705A5788AA0196F4C
:1073400020DAE324CA75A7520C78006269D651840A
:10735000D73770B738B6CC6398CF24118949D7E9AD
:10736000B7DE2F494C85042BD350593391B795A3E1
:10737000809F0F0D003B0F1561894F9C7AC2685D9D
:10738000A6585813D2ADADED354857410C466B1297
:107390000B731344067F773066C10679D1A668E285
:1073A00039756B52DBE3F94E881486D39783210F2E
:1073B000824F596B6FD320797100295DB838587BA3
:1073C000B33DA6CFC6E35B9C1FF9D400C6889C06DC
:1073D0002795FE156706288D2585FE1D48893AFFED
:1073E00009F43693CD5E58F43BBEFA0494B5A44C30
:1073F000062C1884667E51CAC4A2C2F276E1600CE3
:1074000014E1A92DC631982635BFE02C5476A4DAB4
:10741000C79969F7E031B0A8D4B61759CC90995EF6
:10742000E843A586A8A79C79DBE233EDCF85F84336
:10743000A9CAEA723F60F008E9A7C847B3DCFB8A33
:10744000E6DB1972F0016B43D987B36928F6942CF7
:107450000D2F2B752286FB860953469D510315324D
:107460000B1A1DE6200243E2FC0A0E06385050209B
:1074700080ABB712D46C70B53D4BD772B3713CCDB5
:10748000CD68666E3D974A2865253F87B64ACBB6DC
:1074900078214318281DC65627538E8CD19A76D54D
:1074A000C77E50C7A9C7BD0B5262102D6177B7E0E8
:1074B0003D078CF2174885700D14A3FBA2B5B224CA
:1074C0002725D000F3D2FE29BFF22224A2A4B8AE11
:1074D00064EE0330C9980C31BB93ED5B52C80EDAF1
:1074E000490EC70A2CC0B7AB3F894159AF0E1A3DB0
:1074F0007B6864EAD5E91735822B023A2B59203A8A
:107500003BA89953CE6BE5766BC573C5E7F668AAC1
:10751000C6C12AF2B5A833A31F45A6A28B112E55CA
:10752000AC300DF70FA7181E5C105AA9BA62D2AF83
:107530009BAE7A2A3D64F9E99BF87D6CE37E247763
:107540002E9E3CF7467C4131EEAAA2109263A36BBB
:10755000219FBC7A0D8A2F6708240A344B5255FBB1
:10756000377C8849D3FD9603FF4C14D8EEA37ED513
:10757000E810AB20149147997A2B7E8085FF7075B7
:107580008B5919CBC2BC13D77938FE4A58D8956E9F
:10759000FE478F2A707A07A3C79EFDA4FE2EAFEA8E
:1075A000A257AD1ACE6BB48543CF08FDCC7261D91A
:1075B000A1F5CF2152AF7A2C914897C68754C2AF1C
:1075C000B0289509AE277A0C04550F826A82179B62
:1075D000AF7F8A346A3DF9130AE10F04FAC333C15D
:1075E000D422A9AFFA112B72CECADFA6D66B66538E
:1075F000DE5AF2E3E4DE8DFAB19247BF7AA4702539
:10760000ECFB924BA294C599D57B73096994A06D4C
:10761000846E9999691FCA32443227A8DE3A633AC8
:10762000092A9120F130E03244229FFC22C8FF8DCC
:10763000E213E1AB67CF041A9B473F2AAE4CFF87AA
:10764000A8703454A9BE58BAF81AB302D839B00E8B
:1076500084B5DB1B30B6AD23207DD5DC4B35C85D52
:10766000DC915E31617C69327D529D39DABCD2E9B0
:10767000FEB97709035BF9FEA4CA46853C03D8D25C
:10768000C4D4A65CC9E7B4E5012A605D72B482F592
:1076900073719035CA7EF59430DC1F8B9F2527A42B
:1076A000243AE08BDADED6C105E2E6E99A27A28821
:1076B000C285D230C8E2BC580004A99D8F0A5C99EB
:1076C00041BD0D19CCF487D2ECBD274AACD9BBBA69
:1076D0001242FB423F73ED5B16457BF4D81312DF79
:1076E000C9E5787B25990042EDB57885EE3BB195EB
:1076F000C2E70F60633FB5F4636AADA2795DD882DB
:10770000D9BA823F0CA6AFF9EE7F35AB58A5CA9E19
:1077100078FCC7613158E42B431181F68E764BD348
:10772000C079E08C49E6E37F27D61BF576FA89AC71
:107730004E9824BAD63220F1434F4E5F6213BC3BC1
:10774000ADD5A1F3587369BF653D00CC2D38A0C4F9
:10775000014F1DD8B6852B3C5D08D84B5F595AF3B5
:10776000605012D9029DAF5F28B0B3D89C77001645
:1077700017E33697D35F5D87BAC1B772AFF9FA7F67
:10778000F1876E5C208AF1E9FCA602763CD71A7379
:10779000FEFA75539219BF699DB3E92992318D1193
:1077A000B240C80115C186CED3783D64E527DDDF40
:1077B0001FA6E26AA3F267D488EBA390EB24E3CB85
:1077C0004ECB55994F7A9E6157FD2A6BBAE02B0E2E
:1077D000C0B2B7951A0FAD18315AF5E3396B675A35
:1077E000E58A690BFC97A1FD1D8656C671FE2785AB
:1077F000155531DA04A9ABC36D0661A6035C8DB6DD
:107800007EE9EC999A73643CDA7EA0FEECB3351FF6
:10781000221C731BF8E55ECD55A8E4522F7383B686
:107820006BB47F008E44FA752659BD49DEF78D6E24
:107830005E8081FF63A61830144CBCA5C95BE4B21E
:1078400077649C85CDC654C08FF4BCA03F93578607
:107850002FF02248FF201CE5004FE6DBB7BECFB873
:107860008C99914DC75A2FB8547731241C80A08829
:10787000D7C1CAB4605042340117FF546423515435
:10788000F797EFD0E21E4A0943E65389B9C212D1F5
:1078900024FED872A1BFB152575E92FDE0548A52C5
:1078A0003D15BFEB98B03A153C6F160A51CFE57AFB
:1078B0009F2DA75C6B6FA96FDB1C61BCE8897DD233
:1078C000F9FB274B1EABA18B3C3BEDD5B183F5BD3E
:1078D00097E2C54AA11210C6A990AA89E9B655E156
:1078E000452CADA74A9A933E6F4CA6B1289CC4CDB7
:1078F000A6D5CA7E2C9E29F9E1CEE3C56B0404957A
:1079000032CD66203CBFAF826D46A627F50B3C46C4
:10791000FE43DA3FD059FABE16A7E996482ABB893A
:10792000468689DFAFB2892BB4236A78E0474AC91B
:1079300008558AFA00BCDF5450A997710D58D840F9
:10794000FE85044FE77D51B4C478ECFFDC1392A3AD
:107950004EEE9EBEACA449E4D0EA722324E57BD16E
:107960005F1817A4CD55A36F913D7D8633B0E15AC2
:107970005212A722DE11A84A305BF9542811EA619D
:10798000132294DFA15F11D1041733E45F13A650D3
:1079900001111B6FD59A93CB3A06AFECAF69CFD7E5
:1079A0006A78ECC0B9BAF2A2A51750EBA8E7EE4E80
:1079B000CEFF9FCB8D470932177DA62D39AA473DB3
:1079C000267AD8133C31518E91169C50DD6365ACFC
:1079D000C0A64D6B3EEDB01EDB52BB8E8E03791000
:1079E0005118EBCE4DB59681469BE7725833711412
:1079F0006D8A5E508FB7AEDF92663DF4E0D948CB1A
:107A0000E68E4E3E4E714C64B726DA09D3881FCA03
:107A1000057D1536AEC34936DBD624F3CA9A11E28A
:107A200043A491AE6FD3FC9C7F6D52753F72CED351
:107A3000D23DD278A4761E1B1DEA29AE5AA980A099
:107A40007825D9D6D9A52ECE8BFFF0AE25983DC38B
:107A50002BF55C0F4F39BB80385341EA0C415D1E5A
:107A60009FE484D8F473F4992C2C44DED4BEB6F091
:107A70001370679D7078FF04CEF0AFC9F97FBB3CEF
:107A8000486C2A06BC4C9CEADAFBDEB89BBF13CAE2
:107A900051F2A5A188E33B9C365FF5E180E2349486
:107AA000C42FCBC9BA1943BAB7552659DE14FC3EC8
:107AB000F987E0058C446413A595F58EECAF9DAC79
:107AC000EAEE88CB982C6FC074272DD4850A7B17DB
:107AD0001B20549BA3E79BA703BA6D0B4B67C69073
:107AE00062E8A610E76960A22EEAB42F0CF28E704D
:107AF00008E14922194BF4F8456B359502567D7221
:107B0000F7EE031A27E4161237943838E1C764BC3D
:107B1000C05FF66075F3CFB1C5CCAF18D51F9D1609
:107B20006DB30BEA6D2E68A85F0A5C82920BF515A7
:107B30008CEED1A08DCEB5E31BD5EEF8039776B8C9
:107B4000ACB7A0EA22FE25B9DC1125CB226C36B9F0
:107B5000ED01F1F25FCAA28604F324609359FB5150
:107B60005DE4EE57C76FC2F12579941CA909946AA8
:107B7000DD42D0FB5658783539F62321B08A26D31A
:107B8000FA8B15A32F6419148EC59797991C7B70D7
:107B9000257D8BA6266789743EFC782896765F66DD
:107BA0003ACA0550F8D4DA7897D2BF92F858A5139C
:107BB0006DF98025B2B15FB84E28A3D19494110C11
:107BC00040CA24BAD633AF4C3E6913A4AB761BF53A
:107BD000C0640B829D4FAA03ED47CCEC16E2B9BFFF
:107BE000F7D353F25717E050842856C180C1EB6990
:107BF0008BCEC3B01E2F1EB58784E9497F2938D2AA
:107C0000B316A96EC7C4EDD10E83716803542E322A
:107C1000A7D8580A10E2940BE4C924865B7A270A95
:107C20000A801518689EB5AE10986F3B3A80987D13
:107C3000B3FA20E3B15CC08A0C5DE9F957FED25D6E
:107C40003FB077D08A2066A9172908189CC1C0596F
:107C50006049E7BE939291678555A11B04CA1A72C9
:107C6000A25D16F60304050A08060BFF0209070DBC
:107C7000010C00FF2025692025692025692D256933
:107C800000202025633A256900202020205F5F7CAA
:107C9000002C00610044697370206F66660D0A0055
:107CA000555345520046004700424547494E005251
:107CB000414400442E4D590043005052474D005559
:107CC00053455220202000662020006720200042DB
:107CD0004547494E202020202000524144202020AA
:107CE00000442E4D592020200043202020000D0C60
:107CF000205A363C00000500000003072061703B5D
:107D00000000FFFFFFFF4D000000B43F0000000037
:107D1000000081100000CC3F0000D13F0000CF3FA9
:107D20000000FF00000059080000DB3F0000E53FB5
:107D30000000833F00000000000079060000F73FCC
:107D40000000D13F000003400000000000001907C0
:107D5000000005400000D13F00001140000000007D
:107D60000000B108000013400000D13F0000344083
:107D70000000000000004106000036400000D13F36
:107D800000000F000000F4010000040103010201E3
:107D9000010411040F041704160118010000BF7C30
:107DA0000000C77C0000CB7C0000CF7C0000A77CDB
:107DB0000000DA7C0000E17C0000E97C0000BA7C75
:107DC0000000081C242C4448586C74050205080463
:107DD000080B08040405010504090809040608073E
:107DE0000206020402060106040701030803040C4C
:107DF000080D020C0203020C010C040D010D080D0C
:107E00000408020808070802020704080108040918
:107E10000209010A080B020A0201080A010A040BFE
:107E200001020802041008110210021108100110CA
:107E3000041101120212011302130812080F081292
:107E40000413011304140214011502150814081771
:107E5000081404150115041702170119081A02194C
:107E6000021602190119041A01160816041B021B36
:107E7000081A0818021A041B011B04180818040B1E
:107E800004202020202020202020200000000100AD
:107E90000000A07C0000A57C0000A77C0000A97C5D
:107EA0000000A77C0000AF7C0000B37C0000B87C21
:067EB0000000BA7C000096
:00000001FF
